S1130000340632E9FEFBC601E7E901036FE90104A6
S1130010ECE90105830001EDE901051083000010FE
S11300202F0055AEE901093002AFE90109AE84E6BB
S113003084C12D10260041ECF90109C30001EDE94A
S11300400101E6F9010127C84FBD667510830065FB
S1130050270E1083006E2702200E6FE90103200B88
S1130060C601E7E901042003BD02D9ECE90101C39B
S11300700001EDE9010120CAE6E901044F3406E676
S1130080E90105BD00B432628E95431F10BD6501C0
S1130090CC0100340630621F10BD69C03262108387
S11300A000002603BD02E9E6E427DD30E41F10BDAD
S11300B001B220D4340432E9FEFDC601F794EFC640
S11300C05EF794C1C60AF79590C623F794C07F944F
S11300D0BF7F94BEC60DF794BDC605F794BCC60198
S11300E0F794B9C67EF794BBC626F794BACC00053C
S11200F0FD965DF6C843F7969BCC6DB634068E2D
S11300FF95431F10BD65FB32627F92977F92B0CC00
S113010F04B0FD9558C605F794C27F94F37F958D7F
S113011FC65EF792B2C601F792B1F7958E5F4FFDA7
S113012F94EBBD658FFD94D7FF94D5FD94DBFF94BD
S113013FD95F4FFD94E7BD658FFD94CFFF94CDFD3F
S113014F94D3FF94D1C613F792AEC611F792ADCCE8
S113015FFFFFFD950F7F94F07F9664BD11AACCE04D
S113016F04FD92B5CCE000FD9507CC00013406FCEC
S113017F9507BD3A533262CC6DC1BD6501CC6DDBC1
S113018FBD6501CC6DE1BD6501E6E90103270FE60D
S113019FE901074F3406CC0001BD0F57326232E933
S11301AF0104393406327E8E96673410EC64BD0B2D
S11301BF233262ED7E102700F77F96915FF794F15B
S11301CFF792ACCC0008FD950D7F9657C605F794B2
S11301DFC4F694BC4F3406CC10CCBD56E5BD658F28
S11201EFFD94CBFF94C98E6AD73410FC9667BD7C
S1136D5473656E64007265636569766500636F6E5E
S1136D646E65637400676574007365740073686F9B
S1136D7477007365727665720068656C7000657877
S1136D8469740071756974006279650066696E6975
S1136D947368007472616E736D697400666C6578EF
S1136DA400737461746973746963730074616B65EB
S1136DB400004B65726D69742D30393E004B4552A9
S1136DC44D495420464C4558203638303920766590
S1136DD47273696F6E20005620332E31000A0A0044
S1136DE4416D626967756F757320636F6D6D616E54
S1136DF46400556E6B6E6F776E20636F6D6D616E9C
S1136E04640055736167653A204B45524D495420DB
S1136E142D6E202044697361626C65207374617201
S1136E2474757020636F6D6D616E642066696C6542
S1136E340A00202020202020202020202020202080
S1126E442D6520204563686F2073746172747527
S1136E537020636F6D6D616E642066696C650A00F2
S1136E632578004E6F2073756368206C696E652006
S1136E73617661696C61626C65004E6F206C696E4A
S1136E836520746F20636F6E6E65637420746F077F
S1136E9300436F6E6E65637465642E2E2E0A000DB7
S1136EA30A000D0A5965732C2049276D20737469F0
S1136EB36C6C20686572652E2E2E0D0A000D0A4C2B
S1136EC36F6767696E672073757370656E64656455
S1136ED30D0A000D0A4C6F672066696C652069739F
S1136EE3206E6F74206F70656E0D0A000D0A4C6F6F
S1136EF36767696E6720726573756D65640D0A0053
S1136F030D0A4C6F672066696C65206973206E6F88
S1136F1374206F70656E0D0A000D0A4C6F6720664E
S1136F23696C65207374617475733A20006F7065BE
S1136F336E0D0A00636C6F7365640D0A004C6F6712
S1126F4367696E67207374617475733A20200058
S1136F526F6E0D0A006F66660D0A000D0A417267B4
S1136F62756D656E747320617661696C61626C65BE
S1136F723A0D0A0A003F202D2053686F7720746867
S1136F8269732068656C70206D6573736167650D44
S1136F920A0030202D205472616E736D6974204E84
S1136FA2554C4C0D0A0042202D205472616E736DB3
S1136FB269742027425245414B270D0A0043202D74
S1136FC220436C6F736520636F6E6E656374696FC3
S1136FD26E0D0A0048202D205265706F7274206174
S1136FE27661696C6162696C6974790D0A00512079
S1136FF22D2051756974206C6F6767696E6720284C
S113700269662073746172746564290D0A005220E2
S11370122D20526573756D65206C6F6767696E67A5
S11370220D0A0053202D2053686F77207374617406
S11370327573206F6620636F6E6E656374696F6E1D
S11270420D0A00446973636F6E6E656374656451
S11301FE0BCD3262EDE4108300002609CC6DE4BD14
S113020E0D471600A0ECE41083FFFF2609CC6DF613
S113021EBD0D4716008FECE48300011083000F1010
S113022E2200828E023858496E9B0258025E026486
S113023E026A02700276027C028202880288028EB0
S113024E02930298029D02A202A7BD33981600558E
S113025EBD2B2D16004FBD02F0160049BD2B9D1669
S113026E0043BD214416003DBD27EC160037BD07E3
S113027E9B160031BD417C16002BBD02E9160025EC
S113028EBD0A412020BD0A02201BBD0E522016BD00
S113029E10192011BD1086200CCC000134065F4FBE
S11302AEBD0F573262FC950BBD4B8FCCFFFFFD95F6
S11302BE0BF6969227127A9692F69692584F8E963F
S11302CE67EC8BBD5B2F20E9326439CC6E06BD65BD
S11302DE01CC6E36BD6501BD49BF39BD3D58BD4922
S11202EEBF39327C7F7F0AFC9507EDE4F69692C8
S11302FDC101102300498E95073410CC6E6334066A
S113030D8E9667EC02BD65AA32645F4F3406FC9588
S113031D07BD3A533262108300002620CC6E66BDB1
S113032D0D47ECE4FD95071083FFFF270C5F4F3459
S113033D06FC9507BD3A5332623264397F94F0F668
S113034D94F02709CC6E7DBD0D47326439BD3B0257
S113035DCC6E94BD6501C601F792ACFC9507BD3C0E
S113036DFFF692B02705C601F792AF8E7F0FBF7FC0
S113037D0D6F63F692AC102702E8FC92B5BD3CA25A
S113038DED7E1027028CFC92B5BD3CAB8400C47F7E
S113039DE762F192B210270006E66310270243E6E6
S11303AD6353E7635D26CCE662F192B22630FC9589
S11303BD073406E6644FBD3CC93262F692B110268D
S11303CDFFB1FC92B53406E6644FBD3CC932625FA1
S11303DD4F3406E6644FBD06A5326216FF95E662FC
S11203EDC47F4FBD66751083003027371083001F
S11303FC3F1027014C1083006227381083006327B9
S113040C3B108300681027004A10830071102700EA
S113041C56108300721027007E108300731027007F
S113042CA81601B9FC950734065F4FBD3CC932626E
S113043C16FF41FC9507BD3D1316FF387F92AC5F48
S113044C4F3406CC6EA23406FC92B5BD3BB8326474
S113045C16FF215F4F3406CC6EA53406FC92B5BD55
S113046C3BB8326416FF0DF692B027177F92AF5F3C
S113047C4F3406CC6EC03406FC92B5BD3BB8326426
S113048C16FEF15F4F3406CC6ED63406FC92B5BD25
S113049C3BB8326416FEDDF692B02719C601F7920A
S11304ACAF5F4F3406CC6EEF3406FC92B5BD3BB84F
S11304BC326416FEBF5F4F3406CC6F033406FC92D5
S11304CCB5BD3BB8326416FEAB5F4F3406CC6F1C23
S11304DC3406FC92B5BD3BB83264F692B027135F78
S11204EC4F3406CC6F303406FC92B5BD3BB832AA
S11304FB6420115F4F3406CC6F373406FC92B5BDC4
S113050B3BB832645F4F3406CC6F403406FC92B573
S113051BBD3BB83264F692AF27145F4F3406CC6FF1
S113052B523406FC92B5BD3BB8326416FE475F4F9E
S113053B3406CC6F573406FC92B5BD3BB832641607
S113054BFE335F4F3406CC6F5D3406FC92B5BD3B76
S113055BB832645F4F3406CC6F773406FC92B5BD6A
S113056B3BB832645F4F3406CC6F943406FC92B5BF
S113057BBD3BB832645F4F3406CC6FA83406FC9293
S113058BB5BD3BB832645F4F3406CC6FBF3406FC49
S113059B92B5BD3BB832645F4F3406CC6FD634068C
S11305ABFC92B5BD3BB832645F4F3406CC6FF0346C
S11305BB06FC92B5BD3BB832645F4F3406CC701069
S11305CB3406FC92B5BD3BB832645F4F3406CC7035
S11305DB253406FC92B5BD3BB8326416FD97BD12AB
S11205EB5E16FD91FC95073406E6644FBD3CC9CE
S11305FA3262F692B11026FD7DFC92B53406E664A9
S113060A4FBD3CC932625F4F3406E6644FBD06A54E
S113061A326216FD61FC9507BD3CA2ED7E272AFCD9
S113062A9507BD3CABE762FC92B53406E6644FBD60
S113063A3CC932625F4F3406E6644FBD06A5326296
S113064ACC0320FD92B316FD2DF67F0A1027FD2652
S113065AFC92B3830001FD92B3ED7E1026FD17BD13
S113066A073816FD11CC00013406E6644FBD06A511
S113067A3262CC7045BD6501BD3B22ECE4FD9507B1
S113068A1083FFFF2608C601F794F03264395F4FDE
S113069A3406FC9507BD3A533266393404EC6327B1
S11306AA06BD0738326139F692AF1027007DF692FB
S11306BAB010270076E6E4C10D1027006EC10A26A1
S11306CA04C60DE7E4E6E4C1082704C17F2611FC49
S11306DA7F0D10837F0F2312830001FD7F0D200AF3
S11206EAE6E4BE7F0DE780BF7F0D8E7F0F1F10EC
S11306F9C3130410B37F0D261CFC95073406F69228
S1130709AE4FBD3CC93262C601F77F0ACC0320FD56
S113071992B33261398E7F0F1F10C3138810B37FD0
S11307290D2609FC7F0D830001FD7F0D32613932ED
S11307397E8E7F0FAFE4F692B010270053ECE410DD
S1130749B37F0D272DFC7F0B3406AE62E680AF62C2
S11307594FBD636432621083FFFF26E1CC7054BD40
S11307690D47FC7F0BBD4B8F7F92B05FF792AF7F34
S113077992978E7F0FBF7F0DF67F0AC10126117FE5
S11307897F0AFC95073406F692AD4FBD3CC9326227
S1130799359032E8CB7F96597F9658BD128DCC009F
S11307A91434065F4FBD12893262CC707EBD650177
S11307B9CC70B4BD6501BD1609BD3B02CC00013442
S11307C9068E959134103064341030671F10BD19AA
S11307D9CC326610830000102701E610830045100F
S11207E9270209108300471027012310830049BA
S11307F8102700871083004E102701F11083005240
S1130808102700BB10830053270B108300541027B4
S113081801781601B5BD128DE6E4F79659E6614FE5
S113082834068E95911F10BD14FA3262306134106B
S11308388E95911F10BD14853262CC000134068E4A
S113084895913410E6654F3406F696593406CC0073
S113085859BD16C33268F69658F7958F7F96587F18
S1130868955BF69659CB018640BD4541F796597C70
S11308789691CC0046BD2D1E160172BD128DE6E47C
S1130888F79659E6614F34068E95911F10BD14FAF8
S11308983262306134108E95911F10BD1485326216
S11308A8CC000134068E95913410E6654F3406F673
S11308B896593406CC0059BD16C3326816012E6FFA
S11308C862E6624F3063308B3410E6644F8E959144
S11308D8E68BE7F1E6626C624F8E9591E68BC10078
S11208E82706E662E16125D9E6624F3063308B63
S11308F76F84C602F796923063CE9667AF42CC00F8
S113090701BD3D597C94F1BD33F07F96591600DE45
S1130917BD128DF69591C14610270036C14C2703A9
S113092716005FCC000134065F4F34063406E666D2
S11309374F3406CC0059BD16C33268CC70DD34067B
S1130947CC001734065F4FBD126A3264BD3B22BD2B
S113095702E9CC000134065F4F34063406E6664FDD
S11309673406CC0059BD16C33268CC70DE3406CCCD
S1130977001734065F4FBD126A3264BD3B2232E86A
S11309873539CC0001BD0D6F160063F6965727184D
S1130997CC70DF3406CC001734065F4FBD126A32C1
S11309A764BD3B2232E83539CC000134065F4F344D
S11309B7063406F696594F3406CC004EBD16C3329C
S11309C768202BCC0002BD0D6F2023F696572718FD
S11309D7CC70E03406CC001734065F4FBD126A3280
S11209E764BD3B2232E83539CC0001BD0D6F7F72
S11309F694F15FF79691BD160916FDC3F694F02798
S1130A0607CC70E1BD0D4739CC0046BD0A96ED7E94
S1130A162614CC70F73406CC001034065F4FBD1292
S1130A266A3264BD125ECC71063406CC00173406F5
S1130A365F4FBD126A3264BD3B2239F694F0270734
S1130A46CC7107BD0D4739CC004CBD0A96ED7E2608
S1130A5627CC711D3406CC001034065F4FBD126AD4
S1130A663264CC71293406CC001734065F4FBD12AC
S1130A766A3264BD125E2014CC712A3406CC001787
S1130A8634065F4FBD126A3264BD02E9BD3B2239AA
S1130A963404327D7F96597F9658BD128DBD160952
S1130AA6BD3B02E663F795916F61CC000134068E77
S1130AB6959134103406E6674F3406CC0047BD16CC
S1130AC6C33268CC000134068E95F4341030653494
S1130AD61030661F10BD19CC3266108300452714EA
S1120AE610830054271B108300592702201DCCB6
S11370512E0A004572726F722077726974696E67C5
S1137061206C6F672066696C65202D2D206C6F671D
S113707167696E672073746F70706564005365721D
S11370817665722072756E6E696E672E2E2E20548F
S113709179706520796F7572206B65726D697420E2
S11370A12742594527206F72202746494E495348A4
S11370B1270A00636F6D6D616E64732C206F7220FB
S11370C16374726C2D5820746F2071756974207407
S11370D16865207365727665722E0A0000000000EF
S11370E14E6F7420616C6C6F776564206966205201
S11370F1454D4F54450046696E6973682066616960
S11371016C65640A00004E6F7420616C6C6F776566
S1137111642069662052454D4F54450042796520EB
S11371216661696C65640A000000546F6F206D61CB
S11371316E7920636F6D6D616E6420706172616D33
S1127141657465727300257300466174616C2078
S1130AF500013264398E95F41F10BD0E2A5F4F3202
S1130B056439F6965727055F4F326439F696587C53
S1130B159658F195901023FF905F4F32643934064F
S1130B2532E9FF7C7F9692ECE90084EDE4E6F4106B
S1130B3527008DF69692C114260DCC712BBD0D4759
S1130B455F4F32E9008639E6F44FBD57EFED7E2756
S1130B5509ECE4C30001EDE420ED30643410CC71FC
S1130B65473406EC64BD65AA326430641F10BD6663
S1130B7517C30001BD5A77ED62108300002609CC26
S1130B85714ABD0D47BD02E930643410EC64BD659E
S1130B95FB3262F696927C9692584FAEE900883005
S1130BA58BEC62ED84E6F44FBD57EFED7E1026FF26
S1130BB57CE6F41027FF76ECE4C30001EDE420E5C0
S1130BC5CC000132E9008639340632766FE45F4F92
S1130BD5ED64ED66ED68EC6ABD0D31E6E458584FF9
S1120BE5AE6EE69B5D102700CAEC6A3406E6622A
S1130BF458584FAEE810EC8BBD0CD43262ED621041
S1130C0483FFFF2611E6E458584FE36E8E0002304A
S1130C148BEC84326C39EC621027009310A3662F9A
S1130C240CED66E6E44FED64CC0001ED68E6E4E720
S1130C34616C61E66158584FAE6EE69B5D10270007
S1130C4453EC6A3406E66358584FAEE810EC8BBD97
S1130C540CD43262ED621083FFFF2611E66158580A
S1130C644FE36E8E0002308BEC84326C39EC6210EC
S1130C7427FFBE10A3662F0CED66E6E44FED64CCAB
S1130C840001ED68EC6210A3661026FFA45F4FED2B
S1130C946816FF9DEC6826055F4F326C39EC645886
S1130CA4495849E36E8E0002308BEC84326C396C03
S1130CB4E416FF28EC642606CCFFFF326C39EC649E
S1130CC458495849E36E8E0002308BEC84326C39F7
S1130CD43406327C5F4FEDE4EC68BD6617ED62E6E2
S1120CE4F804272DAE64E680AF64AE683001AF2C
S1130CF368E11F270EEC622605ECE43266395F4F88
S1130D033266396C6126026CE4EC62830001ED62A5
S1130D1320CECCFFFF3266393406E6F4270EE6F420
S1130D234FBD6690AEE4E780AFE420EE3590340621
S1130D33E6F4270EE6F44FBD6675AEE4E780AFE450
S1130D4320EE35903406EC6C3406EC6C3406EC6C13
S1130D533406EC6C3406EC6C3406EC6ABD632E3258
S1130D636ACC7168BD632EBD125E3590340632E9D8
S1130D73FF5F8E9543341030621F10BD65FB3262F2
S1130D83CC71F4340630621F10BD65BC3262ECE9E9
S1130D9300A158498E6B1BEC8B340630621F10BDC7
S1130DA365BC3262ECE900A1108300022F3CECE93C
S1130DB300AF3406ECE900AF3406ECE900AF3406C7
S1130DC3ECE900AF3406ECE900AF3406ECE900AF1C
S1130DD3340630E85C1F10BD6598326C30E850343B
S1120DE31030621F10BD65BC326230E41F10BDBA
S11371506572726F7220616C6C6F636174696E67C3
S1137160206D656D6F7279000A0041626F727465FB
S113717064206279207573657200556E696D706C58
S1137180656D656E746564207365727665722063DF
S11371906F6D6D616E64005061636B657420657220
S11371A0726F7200464C4558206572726F72207778
S11371B0726974696E6720646174612C20657272EF
S11371C06F72206E756D6265722069732000436171
S11371D06E6E6F74206372656174652066696C6598
S11371E0200043616E6E6F74206F70656E20666957
S11371F06C6520003A20004572726F723A20257344
S11372000A004B65726D69742061626F7274696EF5
S113721067207769746820666F6C6C6F77696E6736
S1137220206572726F722066726F6D2072656D6F69
S1137230746520686F73743A0046696C6573706591
S11272406320726571756972656400720045722E
S1130DF26617E7E900A0F694C74F34063062341050
S1130E02E6E900A44F3406F696593406CC0045BDF3
S1130E1216C3326830E43410CC71F7BD632E3262EB
S1130E22BD125E32E900A3393406CC72023406CC18
S1130E32001234065F4FBD126A3264ECE43406CC0D
S1130E42001334065F4FBD126A3264BD125E3590E0
S1130E5232E8E8F69692C101220ACC7239BD0D47F6
S1130E6232E818398E9667EC02340630641F10BDDE
S1130E7265FB326230621F10BD124ECC724B3406D7
S1130E8230641F10BD510A3262EDE41083FFFF2665
S1130E920E30623410CC724DBD0D4732E81A39EC73
S1130EA2E4BD525EEDE8161083FFFF1027009DF6A5
S1130EB294F22723FC92B53406ECE818BD3CC932FF
S1130EC262ECE8161083000A260DFC92B53406CCB7
S1130ED2000DBD3CC93262FC9507BD3CA2ED7E10FB
S1120EE227003BF692AE4F3406FC9507BD3CABA0
S1130EF110A3E1262AFC9507BD3CA2ED7E260FF640
S1130F01965727F1CC725EBD650132E81839F69225
S1130F11AD4F3406FC9507BD3CAB10A3E126D6F6D4
S1130F219657270ACC7260BD650132E81839ECE89E
S1130F31161083000A2606CC000DEDE816FC950771
S1130F413406ECE818BD3CC9326216FF53ECE4BD2B
S1130F514B8F32E81839340432E9FECBE6E9013526
S1130F612712CC7262340630E901051F10BD65FBFE
S1130F7132622024F69692C101220BCC726DBD0D12
S1130F814732E90136398E9667EC02340630E901BD
S1130F91051F10BD65FB326230E901031F10BD124C
S1130FA14ECC727F340630E901051F10BD510A325F
S1130FB162EDE41083FFFF10270044ECE43406CC17
S1130FC10100340630661F10BD69613264ED7E276D
S1130FD124E6E90139270F8E95431F10BD650130C1
S1120FE1621F10BD6501E662C10A27CF30621F8F
S1136AD76D5400016D5900026D6100036D69000476
S1136AE76D6D00056D7100066D7600076D7D0008FC
S1136AF76D8200096D87000A6D8C000B6D90000C88
S1136B076D97000D6DA0000E6DA5000F6DB0001000
S1136B176DB50000716A717A719771A471CE71E2D3
S1136B27436861726163746572732073656E743A46
S1136B370909256C640A0044617461206368617201
S1136B476163746572732073656E743A0909256C01
S1136B57640A004E414B27732073656E743A090922
S1136B670925640A005061636B6574732073656E4D
S1136B77743A09090925640A0043686172616374F8
S1136B876572732072656365697665643A090925D8
S1136B976C640A00446174612063686172616374A0
S1136BA76572732072656365697665643A09256C55
S1136BB7640A004E414B27732072656365697665E5
S1126BC7643A09090925640A005061636B657417
S1130FF010BD01B220C6ECE4BD4B8F32E901363995
S1131000E6E90135260E30E901033410CC7281BDC6
S11310100D47326232E9013639327AF69692C101CD
S1131020220CCC729BBD632EBDCD1B16004CCCC0D4
S113103080FDCC14EDE4CC0001ED64F696924F10E3
S1131040A3642F2EEC6458498E9667EC8BED62E610
S1131050F802270EAE62E680AF62AEE4E780AFE44A
S113106020EDC620AEE4E780AFE46C6526026C6434
S113107020C9C60DAEE4E782AFE4BDCD4BCC72B05F
S1131080BD6501326639CC72B2BD632EFC94E3FEB9
S113109094E1340634408E6B271F10BD632E3264F6
S11310A0FC94FDFE94FB340634408E6B3E1F10BD51
S11310B0632E3264FC950534068E6B5A1F10BD6393
S11310C02E3262FC950334068E6B6C1F10BD632EAA
S11310D03262FC94DFFE94DD340634408E6B801F54
S11210E010BD632E3264FC94F9FE94F734063489
S11310EF408E6B9B1F10BD632E3264FC950134063A
S11310FF8E6BBA1F10BD632E3262FC94FF34068EC2
S113110F6BD01F10BD632E3262CC72D2BD632EFC26
S113111F94DBFE94D9340634408E6B271F10BD63C5
S113112F2E3264FC94D7FE94D5340634408E6B3E35
S113113F1F10BD632E3264FC94EB34068E6B5A1F62
S113114F10BD632E3262FC94E934068E6B6C1F1053
S113115FBD632E3262FC94D3FE94D1340634408E98
S113116F6B801F10BD632E3264FC94CFFE94CD347C
S113117F0634408E6B9B1F10BD632E3264FC94E7C4
S113118F34068E6BBA1F10BD632E3262FC94E534A5
S113119F068E6BD01F10BD632E359032785F4FEDE6
S11311AFE4ECE410830100102C005C5F4FED64EC61
S11311BFE4ED665F4FED62EC62108300082C32ECB5
S11311CF648400C4FFA866E8678400C401ED7E2729
S11211DF0CEC6444568884C808ED642006EC6464
S11311EE4456ED64EC664456ED666C6326026C62FE
S11311FE20C6ECE458498E92B7308BEC64ED846CC7
S113120E6126026CE416FF9A3268395F4FFD94B77B
S113121E393404FC94B71F891D8400C4FF3406FCC2
S113122E94B78400C4FF3406E6644FA8E0E8E0589F
S113123E498E92B7EC8BA8E0E8E0FD94B7326139A1
S113124E3406F6CC49C1602605ECE4BD0D1B359081
S113125EF694F02606CC0007BD64FB393406F694EA
S113126EF02616EC643406EC62BD12893262CC723E
S113127EF6BD6501EC66BD650135903406359039D1
S113128E3406EC643406EC62BD12893262E667C041
S113129E41C119102200CC4F8E12AD58496E9B12CB
S11312AEE112F1130113111371132113711371133D
S11312BE71137113711371137113711371137113FC
S11312CE711331134113511371137113711371137C
S11212DE7113618E6BE734108E6C691F10BD1392
S11312ED813264398E6BF434108E6C691F10BD130A
S11312FD813264398E6C0134108E6C691F10BD13EC
S113130D813264398E6C0E34108E6C691F10BD13CE
S113131D813264398E6C1B34108E6C691F10BD13B1
S113132D813264398E6C2834108E6C691F10BD1394
S113133D813264398E6C3534108E6C691F10BD1377
S113134D813264398E6C4234108E6C691F10BD135A
S113135D813264398E6C4F34108E6C691F10BD133D
S113136D813264398E6C5C34108E6C691F10BD1320
S113137D813264393406F694F2C1012524F694F0D1
S113138D261FEC6E3406EC6E3406EC6E3406EC6EF1
S113139D3406EC6E3406EC6E3406EC6CBD632E3202
S11313AD6CF694F2C1022624EC6E3406EC6E34060F
S11313BDEC6E3406EC6E3406EC6E3406EC6E3406CC
S11313CDEC6C3406FC950FBD51D2326E359034065B
S11213DDF694F2C1022624EC6E3406EC6E34064C
S11313ECEC6E3406EC6E3406EC6E3406EC6E34069D
S11313FCEC6C3406FC950FBD51D2326E359034062C
S113140CECE4BD6617C3FFFF3406EC62E3E1EDE4E4
S113141CE6F44FBD57C5ED7E2710E6F4C139260618
S113142CC630E7F435906CF43590AEE4E682AFE464
S113143CC12E261BECE4C30001EDE4C630AEE4304F
S113144C01AFE4E784AEE43001AFE46F843590C6B9
S113145C30AEE43001AFE4E78435903406ECE42795
S113146C0DF696924F10A3E42D045F4F3590CC7279
S113147CF8BD0D47CC000135903406F694C1CB2051
S113148CE7F4F694BCCB20AEE4E701F694BFCB2092
S113149CAEE4E702F694BEC840AEE4E703F694BDAE
S11314ACCB20AEE4E704F694C0AEE4E705F694C6AC
S11314BCAEE4E706C1002608C64EAEE4E706200DEE
S11314CCF694C2C1032306C659AEE4E706F694C7E4
S11214DCCB30AEE4E707F694C5AEE4E708C100F1
S11314EB2606C620AEE4E708C609E7F804359034AF
S11314FB06327FE666C100230AE6F801CBE0F794D7
S113150BC32005C650F794C3E666C101230BAE6135
S113151BE601CBE0F794C42005C605F794C4F69412
S113152BC44F3406CC10CCBD56E5BD658FFD94CBB2
S113153BFF94C9E666C102230BAE61E602CBE0F76A
S113154B94F420037F94F4E666C103230BAE61E6A7
S113155B03C840F794F620037F94F6E666C1042390
S113156B0BAE61E604CBE0F794F52005C60DF794BA
S113157BF5E666C1052309AE61E605F794C82005B7
S113158BC623F794C8E666C10610230030AE61E6A5
S113159B06E7E4C14E26057F94C62024E6E4C15930
S11315AB2614F694C2C1032208F694BAF794C62003
S11315BB0F7F94C6200AE6E4F794C620037F94C6F3
S11315CBE666C1072312AE61E607CBD0E7E4F194DC
S11215DBB92605F794C72005C601F794C7E6663D
S113724F726F72206F70656E696E67202573000A06
S113725F000A004B45524D49542E494E4900466988
S113726F6C6573706563207265717569726564000E
S113727F72004572726F72206F70656E696E67204F
S113728F257320617320696E70757400456E746583
S113729F7220464C455820636F6D6D616E643A20C1
S11372AF000A00546F74616C7320666F72207468E7
S11372BF65206C617374207472616E736665723AC3
S11372CF0A0A000A546F74616C732073696E6365E4
S11372DF204B45524D49542077617320737461726A
S11372EF7465643A0A0A000A0053796E746178204F
S11372FF6572726F72005061636B65742074726192
S113730F6E736D69747465643A2025642C20547906
S113731F70653A2025632C204C656E6774683A209B
S113732F25640A005061636B6574207472616E7317
S112733F6D69747465643A2025640A005479708A
S11315EAC1082315AE61E608E7E4F194BB260AC1F3
S11315FA202706F794C53263397F94C5326339F6D6
S113160A94BDF794F5F694C0F794C8F694BFF7948A
S113161AF4F694BEF794F6F694BCF794C4F694BA26
S113162AF794C6F694BBF794C5F694B9F794C739F8
S113163A39CC0000CE0000FD94F9FF94F7FD94DF45
S113164AFF94DDFD94FDFF94FBFD94E3FF94E15FB9
S113165A4FFD94FFFD9503FD9501FD9505FD94ED60
S113166A39327EFC94E3FE94E18E94D9BD581DFC74
S113167A94FDFE94FB8E94D5BD581DFC94EBF39512
S113168A05FD94EBFC94E9F39503FD94E9FC94DFDE
S113169AFE94DD8E94D1BD581DFC94F9FE94F78E08
S11316AA94CDBD581DFC94E7F39501FD94E7FC9491
S11316BAE5F394FFFD94E53590340432E88EE6E8C8
S11316CA784F3406E6E8743406E6E87A3406CC73CE
S11216DA05BD13DB3266F694F0260EE6E8764F74
S11316E93406CC7333BD632E3262F694F2102700AC
S11316F952F694F2C1012518F694F02613E6E87817
S11317094F3406E6E8743406CC734BBD632E326459
S1131719E6E878272E4FAEE879308B6F84F694F299
S1131729C1012512F694F0260DECE8793406CC7340
S113173960BD632E3262ECE8793406CC7378BD134C
S1131749DB3262FC9503C30001FD95033062AFE807
S113175970F694F44F34068E94F63410FC9507BD54
S11317693BB83264BD1219F694EFAEE870E780AF66
S1131779E870E6E878EBE87CCB22AEE870E780AF66
S1131789E870E6E878EBE87CCB224FEDE868E6E818
S113179978EBE87CCB224FBD121FE6E876CB20AE6E
S11317A9E870E780AFE870E6E876CB204F3406ECC2
S11317B9E86AE3E1EDE868E6E876CB204FBD121F5D
S11317C9E6E872AEE870E780AFE870E6E8724F3495
S11217D906ECE86AE3E1EDE868E6E8724FBD125A
S11317E81FEDE866E6E872C14E2609FC9505C300BC
S11317F801FD95055F4FEDE4E6E8784F10A3E42F6B
S113180835ECE879AEE4E68BAEE870E780AFE870D3
S1131818ECE879AEE4E68B4F3406ECE86AE3E1EDF4
S1131828E868ECE879E68B4FBD121FEDE8666C6159
S113183826026CE420C2E6E87CC101262EECE868A6
S11318488400C4C0475647564756475647564756D6
S1131858E3E8688400C43FEDE868C30020EDE86A63
S1131868AEE870E780AFE87016009FE6E87CC10236
S11318782639ECE868475647564756475647564769
S1131888568400C43FC30020EDE86AAEE870E780E0
S1131898AFE870ECE8688400C43FC30020EDE86C4E
S11318A8AEE870E780AFE87016005FE6E87CC10335
S11318B810260056ECE8661F891D475647564756BA
S11318C847568400C40FC30020EDE86AAEE870E709
S11218D880AFE870ECE8664756475647564756C8
S113734E653A202563204C656E6774683A2025647F
S113735E0A0044617461207472616E736D69747491
S113736E65643A20222573220A00446174612074F4
S113737E72616E736D69747465643A20222573228A
S113738E0A00436865636B73756D3A200043686544
S113739E636B73756D3A2000253032780A00253000
S11373AE3278253032780A0025303278253032781A
S11373BE253032780A005061636B65742072656300
S11373CE65697665643A2025642C20547970653A93
S11373DE2025632C204C656E6774683A2025640A58
S11373EE005061636B6574207265636569766564CC
S11373FE3A2025640A00547970653A202563204C9E
S113740E656E6774683A2025640A00436865636B89
S113741E73756D3A2000436865636B73756D3A201E
S113742E00253032780A0025303278253032780A39
S112743E002530327825303278253032780A0034
S11318E7475647568400C43FC30020EDE86CAEE872
S11318F770E780AFE870ECE8668400C43FC300205B
S1131907EDE86EAEE870E780AFE870F694F2102762
S11319170078F694F2C1012506CC7390BD6501CC1D
S1131927739BBD13DBE6E87CC001C1021022005A99
S11319374F8E193F58496E9B194519571971ECE891
S11319476AC3FFE03406CC73A6BD13813262203A22
S1131957ECE86CC3FFE03406ECE86CC3FFE0340644
S1131967CC73ACBD138132642020ECE86EC3FFE076
S11319773406ECE86EC3FFE03406ECE86EC3FFE020
S11319873406CC73B6BD13813266F694F5AEE870AF
S1131997E780AFE870E6E8784FCE00008E94FBBD91
S11319A7581DECE87030623410A3E1340630643417
S11319B710FC9507BD3BB83264F694F12703BD16B6
S11319C73A32E87339340632E8ECCC000134063095
S11219D7E8143410FC9507BD3B483264108300BC
S11319E6012607CC005432E81639E6E812C47FE72C
S11319F6E812F194EF26D45F4FED62EC62102602F2
S1131A0699BD1219CC0001340630E8143410FC9543
S1131A1607BD3B483264108300012607CC005432CC
S1131A26E81639E6E812C47FE7E812F194EF27CB0B
S1131A364FED66E6E8124FBD121FE6E812CBE0E072
S1131A46E81DCBFEE7F814CC0001340630E8143464
S1131A5610FC9507BD3B483264108300012607CC71
S1131A66005432E81639E6E812C47FE7E812F19426
S1131A76EF1027FF864F3406EC68E3E1ED66E6E8EF
S1131A86124FBD121FE6E812CBE0E7F818CC0001AE
S1131A96340630E8143410FC9507BD3B4832641014
S1131AA68300012607CC005432E81639E6E812C44E
S1131AB67FE7E812F194EF1027FF404F3406EC68F5
S1131AC6E3E1ED66E6E8124FBD121FEDE810E6E825
S1121AD612E7E813C14E2609FC9501C30001FD78
S1131AE595015F4FEDE4E6F8144F10A3E4102F00C1
S1131AF55CCC0001340630E8143410FC9507BD3B7A
S1131B05483264108300012607CC005432E81639A4
S1131B15F694F32608E6E812C47FE7E812E6E8122D
S1131B25F194EF271F4F3406EC68E3E1ED66E6E830
S1131B35124FBD121FEDE810ECE81AAEE4308BE647
S1131B45E812E7846C6126026CE416FF99E6F81442
S1131B554FAEE81A308B6F84CC0001340630E8149C
S1131B653410FC9507BD3B483264108300012607F9
S1131B75CC005432E81639E6E81DC101260DE6E825
S1131B8512CBE04FED68ED6E1600DAE6E81DC102F2
S1131B952649E6E812CBE04FED68584958495849BB
S1131BA5584958495849ED6ECC0001340630E814BB
S1131BB53410FC9507BD3B483264108300012607A9
S1131BC5CC005432E81639E6E812CBE04FED6A341E
S1121BD506ECE810E3E1ED6E16008AE6E81DC1A8
S1131BE40310260081E6E812CBE04FED685849580B
S1131BF449584958491F985FED6ECC0001340630AA
S1131C04E8143410FC9507BD3B483264108300018A
S1131C142607CC005432E81639E6E812CBE04FED3F
S1131C246A5849584958495849584958493406EC56
S1131C34E810E3E1ED6ECC0001340630E81434100E
S1131C44FC9507BD3B483264108300012607CC0091
S1131C545432E81639E6E812CBE04FED6C3406EC66
S1131C64E810E3E1ED6ECC0001340630E8143410DE
S1131C74FC9507BD3B483264108300012607CC0061
S1131C845432E81639E6E812C47FE7E812F194EF17
S1131C941027FD69CC0001ED6216FD61E6F8144FCE
S1131CA4CE00008E94F7BD581DFC94FFC30001FDC3
S1131CB494FFE6E81DC1032607ECE810ED66200F47
S1131CC4E6E81DC1022608EC66840FC4FFED66E64F
S1121CD4E81DC101261AEC668400C4C0475647B8
S1131CE3564756475647564756E3668400C43FED66
S1131CF366E6F8144F3406E6E8153406E6F81C34B1
S1131D0306CC73C4BD13DB3266F694F0260EE6F8F4
S1131D13184F3406CC73EFBD632E3262F694F2107F
S1131D232700A9F694F2C1012518F694F02613E6C8
S1131D33F8144F3406E6E8153406CC7404BD632E58
S1131D433264CC7419BD13DBCC7424BD6501E6E89D
S1131D531DC001C10222424F8E1D6258496E9B1D54
S1131D63681D761D88EC683406CC742FBD1381324C
S1131D73622026EC6A3406EC6A3406CC7435BD134F
S1131D838132642014EC6C3406EC6C3406EC6C3451
S1131D9306CC743FBD13813266E6F814272E4FAE8A
S1131DA3E81A308B6F84F694F2C1012512F694F08D
S1131DB3260DECE81A3406CC744DBD632E3262EC66
S1131DC3E81A3406CC7462BD13DB3262F6969127AB
S1121DD303BD163AEC6610A36E27065F4F32E885
S1131DE21639E6E8134F32E8163934063278EC68CD
S1131DF2FD9509F694C7CBFF3404F694C3CBFDE0FA
S1131E02E04FED64E66D270FFC950BBD525EFD7E3F
S1131E12708E7E76BF7E74FC7E7410837E7627205D
S1131E228E7E76BF7E72FC7E7210B37E7427111F83
S1131E3201E680BF7E72BE9509E780BF950920E660
S1131E428E7E76BF7E74FC7E701083FFFF102700A7
S1131E52C7CC0001ED62FC950BBD525EEDE410832C
S1131E62FFFF2728EC621083005E2C20F694C5271E
S1131E721BECE410B37E7026131083000A2605F6C9
S1131E8294F327086C6326026C6220CAEC62108306
S1131E9200012F26108300022608FC7E70BD1F302D
S1131EA22018F694C5BE9509E780BF9509EC62C374
S1131EB20020BE9509E780BF9509EC62BD658F8E4F
S1131EC29695BD581DFC7E70BD1F30ECE4FD7E70FE
S1121ED2FC9509A368ED6610A3642F29FC7E72AA
S1131EE110B3950927111F01E680BF7E72BE7E746F
S1131EF1E780BF7E7420E6FC7E74837E763406EC34
S1131F0168A3E1326A39EC6610A3642603326A39A4
S1131F11FC9509FD7E7216FF2EEC6810B395092617
S1131F2106CCFFFF326A39FC9509A368326A393459
S1131F3106327FEC618400C47FE7E4EC6110830026
S1131F417F2F0DF694C62708BE9509E780BF950932
S1131F51E6E4C1201025001BC17F10270015F19470
S1131F61C81027000EF194C510270007F194C6107C
S1131F7126004EEC611083000A261AF694F3261506
S1131F81F694C8BE9509E780BF9509C64DBE95096B
S1131F91E780BF9509F694C8BE9509E780BF950906
S1131FA1E6E4270FF194C82718F194C52713F19497
S1131FB1C6270EEC618800C840ED61E6E4C840E73D
S1131FC1E4F694F32712F694C6260DE662BE95094B
S1121FD1E780BF9509326339E6E4BE9509E780DE
S1131FE0BF9509326339340632775F4FEDE4EC6D07
S1131FF010A3E4102F0148EC69AEE4E68BE766F128
S113200094C526261F10E3698E0001308BE684CB2D
S1132010E04FED646C6126026CE46C6126026CE4B2
S1132020ECE4AE69E68BE7662005CC0001ED64E6DE
S113203066F194C62614C601E7686C6126026CE456
S1132040ECE4AE69E68BE76620026F68E666F1941D
S1132050C826286C6126026CE4ECE4AE69E68BE7E2
S113206066C47FE7674F1083003F2D0FE6674F106C
S113207083005F2E06E666C840E766E6682706E644
S113208066CA80E766EC64BD658F8E9695BD581D63
S11320905F4FED62EC6210A364102C0099F694F388
S11320A0271BFC950B3406E6684FBD63643262104F
S11320B083FFFF10260076CCFFFF326B39E666C142
S11320C00A10270071C1092630FC950D830001FD1B
S11220D0950D108300002D19FC950B3406CC00E0
S113744D446174612072656365697665643A2022CE
S113745D2573220A0044617461207265636569763F
S113746D65643A20222573220A00646562756700FB
S113747D657363617065006C696E65006261756446
S113748D00636F6E66696775726174696F6E0074FF
S113749D696D656F75740070726F6D7074006669D7
S11374AD6C6574797065006C6F67006475706C65DC
S11374BD780068616E647368616B6500626C6F63FC
S11374CD6B5F636865636B5F74797065007265707B
S11374DD6561745F71756F7465007265747279009E
S11374ED7061636B65745F6C656E67746800706161
S11374FD6464696E670070616463686172007374BB
S113750D6172745F6F665F7061636B657400656E45
S113751D645F6F665F6C696E650071756F7465008D
S113752D65696768745F6269745F71756F7465000E
S112753D696E636F6D706C6574650064656C6175
S11320DF20BD636432621083FFFF26DECCFFFF3224
S11320EF6B39CC0008FD950D2034FC950B3406E6B6
S11320FF684FBD636432621083FFFF2606CCFFFF77
S113210F326B39FC950D830001FD950D1083000092
S113211F2F06E666C10D2606CC0008FD950D6C63EF
S113212F26026C6216FF5E6C6126026CE416FEAF2B
S113213F5F4F326B39327E8E6C6D34108E9667EC36
S113214F02BD0BCD3262EDE4108300002608CC757E
S113215F57BD0D473590ECE41083FFFF2608CC756F
S113216F6FBD0D473590CC0003BD1467ED7E10266F
S113217F00BAECE483000110830017102200AD8E27
S113218F219558496E9B21C521CA21CF21D421D92C
S113219F21DE21E321E821ED21F221F721FC2201A7
S11321AF2206220B22102215221A221F2224222950
S11321BF222E22332238BD223D3590BD22ED35909B
S11221CFBD22F73590BD23473590BD23A0359031
S11321DEBD23D23590BD23F93590BD24203590BD55
S11321EE244E3590BD24F23590BD25203590BD2664
S11321FEDD3590BD25D63590BD26773590BD261597
S113220E3590BD263A3590BD265B3590BD26B0354A
S113221E90BD26833590BD256A3590BD25973590A2
S113222EBD27003590BD272E3590BD273A35903207
S113223E7ECC0002BD2785EDE41083FFFF2719E64F
S113224E61F794F2FC950F1083FFFF2703BD4B8FAC
S113225ECCFFFFFD950F35908E9667E698044FBD23
S113226E66751083006C1026006EF69692C10424D7
S113227E08CC7585BD0D473590FC950F1083FFFF77
S113228E2708CC7597BD0D4735908E9667EC0634AE
S113229E068E95111F10BD65FB32628E9667EC0695
S11322AEBD124ECC75B334068E9667EC06BD510A3C
S11322BE3262FD950F1083FFFF2616F6CC204F34A5
S11222CE068E9667EC063406CC75B5BD0D473207
S11322DD6639C602F794F235905F4FBD1467359099
S11322ED8E9667E69804F792B2398E9667E698044F
S11322FD4FBD667510830072260FBD3D58CCFFFF90
S113230DFD9507C601F794F0398E95073410CC75F9
S113231DE934068E9667EC04BD65AA32645F4F34CA
S113232D06FC9507BD3A533262108300002607CC94
S113233D75ECBD0D47397F94F03932788E6D45AF0C
S113234D668E9667EC04BD44C8EDE45F4FED64EC16
S113235DF8062720AE66EC81AF6610A3E4260CECDC
S113236DF806ED62CC0001ED642009EC66C30002B1
S113237DED6620DBEC642712ECE4FD95585F4F34D9
S113238D06FC9507BD3A53326A39CC7603BD0D4729
S113239D326839327E8E9667EC04BD44C8EDE41084
S11323AD8300002D06108300072F08CC7611BD0D78
S11323BD473590E661F794C25F4F3406FC9507BD2F
S11223CD3A53326439327E8E9667EC04BD44C8AD
S113754C79007761726E696E670000416D626967DC
S113755C756F757320277365742720636F6D6D6168
S113756C6E6400556E6B6E6F776E2027736574278F
S113757C20636F6D6D616E640046696C6573706534
S113758C6320726571756972656400446562756720
S113759C206C6F672066696C6520616C7265616430
S11375AC79206F70656E0077004572726F72206F70
S11375BC70656E696E67206465627567206C6F67B1
S11375CC2066696C652025732C206572726F72209D
S11375DC6E756D62657220697320256400257800D0
S11375EC4E6F2073756368206C696E6520617661DB
S11375FC696C61626C6500496E76616C69642073B8
S113760C7065656400496D70726F70657220766187
S113761C6C756500496D70726F7065722076616C63
S113762C7565004572726F7220636C6F73696E6757
S112763C206C6F672066696C65202573004C6FA6
S11323DCEDE4108300002F06108300642F08CC76E4
S11323EC20BD0D473590E661F794BC35908E966709
S11323FCEC04BD6617108300142F088E9667AE0488
S113240C6F88148E9667EC0434068E95431F10BDAA
S113241C65FB3590327F8E9667E698044FBD6675E2
S113242CE7E4C16126067F94F3326139E6E4C162C4
S113243C2608C601F794F33261395F4FBD14673235
S113244C61398E9667E69804C12D2629F692B02739
S113245C24FC7F0BBD4B8F1083FFFF260D8E9297B0
S113246C3410CC762FBD0D4732627F92977F92AF9A
S113247C5FF792B039F692B02707CC7649BD0D4779
S113248C398E9667EC04BD6617108300142F088EE2
S113249C9667AE046F88148E9667EC0434068E929D
S11324AC971F10BD65FB32628E92971F10BD124EA2
S11324BCCC765F34068E92971F10BD510A3262FDA2
S11224CC7F0B1083FFFF26188E92973410CC7667
S11324DB61BD0D4732627F92977F92AF5FF792B0E7
S11324EB39C601F792B039327F8E9667E698044F5E
S11324FBBD6675E7E4C1662608C601F792B1326181
S113250B39E6E4C16826067F92B13261395F4FBD6B
S113251B1467326139327ECC0004BD1467ED7E1032
S113252B26003A8E9667EC04BD44C8E7E48E9667A2
S113253BEC06BD44C8E761E6E4C100250EC17F2269
S113254B0AE661C1002504C17F2308CC767BBD0D4F
S113255B472005E6E4F792ADE661F792AE3590328B
S113256B7F8E9667E69804E7E44FBD2758ED7E27E8
S113257B18E6E4F194BA270BF194BB2706F794C041
S113258B326139CC7689BD0D47326139327F8E96F3
S113259B67E69804E7E44FBD66901083004E260669
S11325AB7F94BA326139E6E44FBD2758ED7E271884
S11325BBE6E4F194C0270BF194BB2706F794BA32E7
S11225CB6139CC76A2BD0D47326139327F8E96CD
S113764B672066696C6520616C7265616479206F73
S113765B70656E0077004572726F72206F70656E85
S113766B696E67206C6F672066696C6520257300F3
S113767B496C6C6567616C2076616C756500436859
S113768B6172616374657220616C726561647920E7
S113769B696E20757365004368617261637465720A
S11376AB20616C726561647920696E207573650065
S11376BB43686172616374657220616C72656164A5
S11376CB7920696E2075736500496E76616C696407
S11376DB206C656E6774680056616C7565206F75F8
S11376EB74206F662072616E6765002578002578BB
S11376FB00456E64206F66206C696E65206D757332
S113770B7420626520646966666572656E74206FA9
S113771B66207374617274206F66207061636B658D
S113772B74002578005374617274206F6620706145
S112773B636B6574206D757374206265206469D7
S11325DA67E69804E7E44FBD66901083004E26062A
S11325EA7F94BB326139E6E44FBD2758ED7E271844
S11325FAE6E4F194C0270BF194BA2706F794BB32A8
S113260A6139CC76BBBD0D47326139327F8E96670C
S113261AEC04BD44C8E7E4C10A2504C15E2309CC1D
S113262A76D4BD0D47326139E6E4F794C132613993
S113263A327E8E9667EC04BD44C8EDE41083005ED6
S113264A2F08CC76E3BD0D473590E661F794BF3584
S113265A90327E30E43410CC76F634068E9667ECEB
S113266A04BD65AA3264E661F794BE35908E966716
S113267AEC04BD44C8F7959039327E30E43410CC6A
S113268A76F934068E9667EC04BD65AA3264F6942C
S113269AEF4F10A3E42608CC76FCBD0D473590E62F
S11326AA61F794BD3590327E30E43410CC772D3402
S11326BA068E9667EC04BD65AA3264F694BD4F1083
S11226CAA3E42608CC7730BD0D473590E661F7C1
S11326D994EF3590327F8E9667EC04BD44C8E7E4E5
S11326E9C101250AC1032206F794B9326139CC77AD
S11326F961BD0D47326139327F8E9667E698044F82
S1132709BD6690E7E4C14B2608C601F7958D326191
S113271939E6E4C14426067F958D3261395F4FBDA0
S113272914673261398E9667EC04BD44C8FD965D21
S113273939327ECC0002BD2785EDE41083FFFF27E3
S113274907E661F7958E35905F4FBD146735903470
S113275904E6E4C1212504C13E2310E6E4C17B2536
S113276904C17E2306E6E4C1602606CC0001326179
S113277939CC7774BD0D475F4F3261393406ECE4C7
S113278958498E9667EC8BBD0D31CC77863406ECAF
S11327996258498E9667EC8BBD65D232621083000C
S11327A9002605CC00013590CC77893406EC6258B3
S11327B9498E9667EC8BBD65D2326210830000277F
S11227C919CC778C3406EC6258498E9667EC8BEA
S1136BD6732072656365697665643A090925640AF2
S1136BE60041626F7274202020202020200042720F
S1136BF665616B2020202020202000436F6D706C7F
S1136C0665746520202020004461746120202020C2
S1136C16202020200046696C656E616D6520202069
S1136C2620005265636569766520696E6974005350
S1136C36656E6420696E69742020200054696D6550
S1136C466F7574202020202000456E64206F662016
S1136C5666696C652000556E6B6E6F776E2020201A
S1136C6620200025730A0074770001747D000274E5
S1136C7684000374890004748E0005749C000674F1
S1136C86A4000774AB000874B4000974B8000A744D
S1136C96BF000B74C9000C74DA000D74E7000E749F
S1136CA6ED000F74FB001075030011750B001275CF
S1136CB61B001375270014752D0015753D001675F8
S1126CC6480017754E00187556000077900001AE
S113774A66666572656E74206F6620656E64206F66
S113775A66206C696E6500496E76616C69642063A3
S113776A6865636B207479706500496E76616C692B
S113777A6420636861726163746572006F6E006F7E
S113778A66006F666600616C6C006465627567000A
S113779A657363617065006C696E65006261756426
S11377AA00636F6E66696775726174696F6E0074DF
S11377BA696D656F75740066696C657479706500C6
S11377CA6C6F67006475706C65780068616E6473C9
S11377DA68616B6500626C6F636B5F636865636B9A
S11377EA5F74797065007265706561745F71756F35
S11377FA7465007265747279007061636B65745F95
S113780A6C656E6774680070616464696E670070A1
S113781A6164636861720073746172745F6F665F36
S113782A7061636B657400656E645F6F665F6C6933
S112783A6E650071756F74650065696768745FCA
S11327D8BD65D232621083000026045F4F3590CC69
S11327E8FFFF3590327E8E6CD134108E9667EC02E2
S11327F8BD0BCD3262EDE4108300002608CC786D61
S1132808BD0D473590ECE41083FFFF2608CC78868D
S1132818BD0D473590ECE4830001108300171022A6
S113282800AD8E283158496E9B28612866286B288C
S1132838702875287A287F28842889288E28932840
S113284898289D28A228A728AC28B128B628BB28F0
S1132858C028C528CA28CF28D4BD28D93590BD2971
S11328681F3590BD29573590BD29653590BD2984FC
S11328783590BD29913590BD29A53590BD29B3352D
S113288890BD29D43590BD293E3590BD29F33590A6
S1132898BD2AB13590BD2A1D3590BD2A6B3590BD32
S11328A82A793590BD2A953590BD2AA33590BD2A3D
S11328B85D3590BD2A873590BD2A0F3590BD2A3DD8
S11228C83590BD2AE33590BD2AFC3590BD2B0910
S11378496269745F71756F746500696E636F6D70D9
S11378596C6574650064656C6179007761726E6941
S11378696E670000416D626967756F7573202773D0
S1137879686F772720636F6D6D616E6400556E6B59
S11378896E6F776E202773686F772720636F6D6D2E
S1137899616E640044656275673A0909090900461D
S11378A9696C653A2025730A004475706C65783AE9
S11378B9090909090046756C6C0A0048616C660A75
S11378C900457363617065206368617261637465FF
S11378D9723A090925630A004C696E653A0909096E
S11378E9090052656D6F74650A0025780A004261C2
S11378F97564726174653A090909256420626175C0
S1137909640A003720626974732C206576656E20D9
S11379197061726974792C20322073746F702062DB
S1137929697473003720626974732C206F6464204E
S11279397061726974792C20322073746F70201E
S113794862697473003720626974732C20657665E4
S11379586E207061726974792C20312073746F7091
S113796820626974003720626974732C206F646420
S1137978207061726974792C20312073746F7020BF
S1137988626974003820626974732C206E6F2070E9
S113799861726974792C20322073746F7020626963
S11379A87473003820626974732C206E6F207061C0
S11379B8726974792C20312073746F702062697431
S11379C8003820626974732C206576656E207061B6
S11379D8726974792C20312073746F702062697411
S11379E8003820626974732C206F6464207061729B
S11379F86974792C20312073746F70206269740063
S1137A08436F6E66696775726174696F6E3A0909C6
S1137A180925730A0054696D656F75743A09090973
S1137A282564207365636F6E64730A0046696C6528
S1127A38747970653A0909090042696E617279BF
S11328D73590BD2965BD2984BD2991BD2957BD29D9
S11328E7B3BD2B09BD29D4BD293EBD291FBD2AE38C
S11328F7BD29F3BD2A6BBD29A5BD2AFCBD2A5DBD33
S11329072A87BD2A0FBD2A3DBD2A1DBD2A79BD2AA6
S113291795BD2AA3BD2AB139CC789DBD6501F6942E
S1132927F2C10227054FBD2B17398E95113410CCF0
S113293778A8BD632E3590CC78B2BD6501F692B107
S11329472707CC78BEBD650139CC78C4BD6501398C
S1132957F692B24F3406CC78CABD632E3590CC7844
S1132967E1BD6501F694F02707CC78EBBD65013925
S1132977FC95073406CC78F3BD632E3590FC955847
S11329873406CC78F7BD632E3590F694C2584F8E33
S11329976D35EC8B3406CC7A08BD632E3590F694EE
S11329A7BC4F3406CC7A1DBD632E3590F694F34F95
S11329B73406CC7A34BD65013262F694F32707CC2A
S11229C77A41BD650139CC7A49BD650139CC7AB5
S1137A470A0041736369690A004C6F672066696CB1
S1137A57653A0909090025730A004E6F6E650A0025
S1137A6748616E647368616B652073746172743AFC
S1137A77090925642028646563290A0048616E643E
S1137A877368616B652073746F703A200909256404
S1137A972028646563290A0051756F74652063683B
S1137AA7617261637465723A090925630A00526554
S1137AB7706561742071756F7465206368617261A4
S1137AC7637465723A0909004E6F6E650A0025638F
S1137AD70A0045696768742D6269742071756F744B
S1137AE765206368617261637465723A09004E6F59
S1137AF76E650A0025630A005374617274206F6609
S1137B07207061636B65743A09092530322E327827
S1137B172028686578290A004D6178696D756D209C
S1137B27726574727927733A090925642028646594
S1127B3763290A005061636B6574206C656E6787
S11329D650BD6501F69297270D8E92973410CC7AE6
S11329E65DBD632E3590CC7A61BD650139F692AD35
S11329F64F3406CC7A67BD632E3262F692AE4F34FC
S1132A0606CC7A83BD632E3590F694C04F3406CC3B
S1132A167A9FBD632E3590CC7AB5BD6501F694BB1D
S1132A262607CC7ACFBD650139F694BB4F3406CC64
S1132A367AD5BD632E3590CC7AD9BD6501F694BAA4
S1132A462607CC7AF5BD650139F694BA4F3406CC1F
S1132A567AFBBD632E3590F694EF4F3406CC7AFF9D
S1132A66BD632E3590F695904F3406CC7B1FBD631F
S1132A762E3590F694C14F3406CC7B3BBD632E3580
S1132A8690F694BD4F3406CC7B56BD632E3590F636
S1132A9694BF4F3406CC7B7CBD632E3590F694BE32
S1132AA64F3406CC7B97BD632E3590CC7BB9BD6580
S1132AB601F694B9C001C10222224F8E2AC8584990
S1122AC66E9B2ACE2AD52ADCCC7BCCBD65013988
S1137B4674683A09090925642028646563290A00CA
S1137B56456E64206F66206C696E65206368617289
S1137B6661637465723A09092530322E3278202809
S1137B76686578290A0050616464696E6720636FDA
S1137B86756E743A09090925642028646563290A0F
S1137B960050616464696E6720636861726163742E
S1137BA665723A09092530322E32782028686578BC
S1137BB6290A00426C6F636B636865636B20747992
S1137BC670653A0909004F6E6520636861726163E6
S1137BD674657220636865636B73756D0A00547708
S1137BE66F2063686172616374657220636865639C
S1137BF66B73756D0A0054687265652063686172FB
S1137C066163746572204352432D43434954540AB5
S1137C1600496E636F6D706C6574652066696C658A
S1137C2620646973706F736974696F6E3A09004BE7
S1127C366565700A00446973636172640A0044EF
S1132AD5CC7BE4BD650139CC7BFCBD650139CC7C7F
S1132AE517BD6501F6958D2707CC7C35BD65013984
S1132AF5CC7C3BBD650139FC965D3406CC7C44BD7C
S1132B05632E3590CC7C67BD6501F6958E4FBD2B44
S1132B1517393406ECE42708CC7C80BD6501359073
S1132B25CC7C84BD65013590F69692C1022307CC11
S1132B357C89BD0D4739F69692C10226138E966798
S1132B45EC0234068E955B1F10BD65FB32622003D3
S1132B557F955B7C96917F9659BD128DBD3B02FC9A
S1132B659507BD3CFFCC0052BD2D1EED7E2611CC34
S1132B757CA33406CC001034065F4FBD126A326460
S1132B85CC7CB33406CC001434065F4FBD126A32D4
S1132B9564BD125EBD3B2239327EF69692C1012296
S1132BA508CC7CB4BD0D4735907F955BC602F7967E
S1132BB5917F9659BD128DBD3B02C601E761E66161
S1122BC54FBD3D59ED7E270C6F61BD2C07E7E432
S1132BD45D270220EAE6E42611CC7CC93406CC0045
S1132BE41034065F4FBD126A3264CC7CD53406CCF3
S1132BF4001434065F4FBD126A3264BD125EBD3BDD
S1132C04223590327E7F96597F9658BD16097F9659
S1132C1457FC968FBD6617E7E4FC968F34068E95B1
S1132C24911F10BD65FB3262F694F2271ECC7CD64C
S1132C34BD13DBCC7CE6BD6501CC00523406CC006C
S1132C440D3406CC0014BD128E3264FC9507BD3CD1
S1132C54FFCC000134068E95913410E6644F34069B
S1132C64F696593406CC0052BD16C33268CC000122
S1132C7434068E95F434103065341030661F10BD5C
S1132C8419CC326610830045102700681083005362
S1132C94270B108300541027006616006CE6E44FDB
S1132CA434068E95F41F10BD14FA326230E43410E5
S1132CB48E95911F10BD14853262CC000134068EAA
S1122CC495913410E6644F3406F696593406CCD5
S1132CD30059BD16C33268F69658F7958F7F9658F8
S1132CE3F69659CB018640BD4541F79659CC00462B
S1132CF3BD2D1E35908E95F41F10BD0E2A5F4F35E2
S1132D0390F6965727045F4F3590F696587C96585D
S1132D13F195901025FEFB5F4F35903404BD163BAF
S1132D23E6E4C1462703BD1609E6E4F7965A7F96FF
S1132D33587F955A7F9657F694F2271FCC7CF6BD9D
S1132D4313DBCC7D06BD6501F6965A4F3406CC00E1
S1132D530D3406CC0014BD128E3264F6965AC14368
S1132D6310270029C144271CC146270FC15227023B
S1132D732024BD2DA1F7965A16FFBCBD2E7AF796D3
S1132D835A16FFB3BD3140F7965A16FFAABD166B08
S1132D93CC0001326139BD166B5F4F326139327E2B
S1132DA3F696587C9658F195902505C6414F359073
S1132DB3CC000134068E959134103065341030669E
S1122DC31F10BD19CC3266108300001027008446
S1137C45656C6179206265666F72652073656E6423
S1137C55696E673A09092564207365636F6E6473F9
S1137C650A0046696C6520636F6E666C69637420EF
S1137C757761726E696E673A0909004F6E0A004FA3
S1137C8566660A004F6E6C79206F6E652066696CB6
S1137C95656E616D6520616C6C6F77656400526516
S1137CA56365697665206661696C65642E000046C6
S1137CB5696C6573706563287329207265717569CC
S1137CC572656400476574206661696C65642E009D
S1137CD500526563656976652073746174653A203D
S1137CE500526563656963652073746174653A2040
S1137CF500526563656976652073746174653A201D
S1137D0500526563656976652073746174653A200C
S1137D15006277007700720025735761726E696E91
S1137D25673A2046696C6520257320616C7265612C
S1127D356479206578697374732C2063726561B7
S1132DD2108300451027006510830053270B1083CE
S1132DE200541027006416008AE6E44F34068E95D8
S1132DF2911F10BD14FA326230E434108E95911F83
S1132E0210BD14853262CC000134068E95913410C3
S1132E12E6644F3406F696593406CC0059BD16C3FF
S1132E223268F69658F7958F7F9658F69659CB01E5
S1132E328640BD4541F79659C6464F35908E95F466
S1132E421F10BD0E2AC6414F3590F696572705C668
S1132E52414F3590CC000134065F4F34063406F6F8
S1132E6296594F3406CC004EBD16C33268F6965AB4
S1132E724F3590C6414F3590327CF696587C965821
S1132E82F195902506C6414F326439F694C74F3402
S1132E92068E959134103064341030671F10BD19BA
S1132EA2CC3266108300001027026C10830042109B
S1132EB2270219108300451027023E108300461092
S1122EC22700C1108300532713108300541027D7
S1132ED102361083005A1027005F16025CF6958FA4
S1132EE17C958FF195902506C6414F326439F6964B
S1132EF1592604C63F2005F69659CBFFE1E4263353
S1132F01306134108E95911F10BD14853262CC004E
S1132F110134068E95913410E6654F3406E6663425
S1132F2106CC0059BD16C332687F9658F6965A4F9F
S1132F31326439C6414F326439F6958F7C958FF1ED
S1132F4195902506C6414F326439F696592604C632
S1132F513F2005F69659CBFFE1E42623F694C74FAB
S1132F6134065F4F34063406E6664F3406CC005906
S1132F71BD16C332687F9658F6965A4F326439C6E5
S1132F81414F326439E6E4F196592706C6414F327E
S1132F916439F6955B260F8E959134108E955B1FDF
S1132FA110BD65FB32628E955B1F10BD124ECC00C5
S1132FB100CE0000FD9697FF9695F694F32707CC73
S1122FC17D16ED622005CC7D19ED62CC7D1B34AD
S1132FD0068E955B1F10BD510A3262FD950B10835E
S1132FE0FFFF10270041BD4B8FF6958E1027003749
S1132FF0F694F02627CC001234065F4FBD128932B6
S1133000628E955B3410CC7D523406CC7D1DBD633D
S11330102E3264BD125ECC7D53BD65018E955B1F5F
S113302010BD140A16FFA5EC6234068E955B1F10C2
S1133030BD510A3262FD950B1083FFFF26188E9551
S11330405B3410CC7D553406CC0004BD0D6F326466
S1133050C6414F326439CC7D583406CC0002340664
S11330605F4FBD126A32648E955B3410CC0002341B
S113307006CC0014BD126A3264CC7D64BD65018E39
S1133080955B3410CC7D65BD13DB3262FC9507BDC6
S11330903CFFF694C74F34065F4F34063406F69669
S11330A0594F3406CC0059BD16C33268F69658F70A
S11330B0958F7F96587F955A7F9657F69659CB01F0
S11230C08640BD4541F79659C6444F326439E600
S11330CFE4F196592706C6414F326439F694C74F37
S11330DF34065F4F34063406F696594F3406CC0047
S11330EF59BD16C33268C6434F3264398E95911F4A
S11330FF10BD0E2AC6414F326439F69657270B5F1F
S113310F4FBD0D6FC6414F326439F694C74F340625
S113311F5F4F34063406F696594F3406CC004EBD35
S113312F16C33268F6965A4F326439C6414F326429
S113313F39327DF696587C9658F195902506C641FE
S113314F4F326339F694C74F34068E95913410304D
S113315F64341030671F10BD19CC32661083000021
S113316F102701FE10830044272B108300451027DE
S113317F01D2108300461027011810830054102722
S113318F01D010830058102701081083005A10270C
S113319F014C1601EEE6E4F196591027004CF69512
S11331AF8F7C958FF195902506C6414F326339F682
S11231BF96592604C63F2005F69659CBFFE1E446
S11331CE2623F694C74F34065F4F34063406E6665C
S11331DE4F3406CC0059BD16C332687F9658F69606
S11331EE5A4F326339C6414F326339F6955A270B1B
S11331FE5F4FBD0D6FC6414F326339E6614F3406E2
S113320E8E95911F10BD1FE632621083FFFF2619A3
S113321EF6CC204F3406CC7D783406CC0003BD0D9D
S113322E6F3264C6414F326339C601E762F7955A6D
S113323EF696574F108300182607C658F795912017
S113324E19F696574F1083001A260AC65AF7959107
S113325E7F969420056F627F955AF694C74F340675
S113326E8E95913410E6664F3406F696593406CC94
S113327E0059BD16C33268F69658F7958F7F965847
S113328EF69659CB018640BD4541F79659C6444F33
S113329E326339F6958F7C958FF195902506C6414C
S11332AE4F326339F696592604C63F2005F69659D1
S11232BECBFFE1E42623F694C74F34065F4F3469
S11332CD063406E6664F3406CC0059BD16C3326883
S11332DD7F9658F6965A4F326339C6414F32633949
S11332EDE6E4F196592706C6414F326339F694C781
S11332FD4F34065F4F34063406F696594F3406CCD8
S113330D0059BD16C33268FC950BBD4B8FE661C1E8
S113331D01261DCC7D7BBD6501BD125EF69591C167
S113332D44260DF6958D26088E955B1F10BD66C639
S113333D7F955BF69659CB018640BD4541F796596D
S113334DC6464F3263398E95911F10BD0E2AC64164
S113335D4F326339F69657270B5F4FBD0D6FC6413C
S113336D4F326339F694C74F34065F4F3406340633
S113337DF696594F3406CC004EBD16C33268F696F8
S113338D5A4F326339C6414F326339F69692C101B1
S113339D2207CC7D8EBD0D4739CC0001BD3D59EDC5
S11333AD7E2607CC7DA3BD0D47397C94F1BD128DCE
S11233BDBD3B02BD33F0ED7E2611CC7DB5340649
S11333CCCC001034065F4FBD126A3264CC7DC2341B
S11333DC06CC001434065F4FBD126A3264BD125E13
S11333ECBD3B2239BD163BBD1609C653F7965A7F11
S11333FC96597F9658F694F0270EFC965D3406CCBD
S113340C03E8BD56E5BD3D2BFC9507BD3CFFF6948A
S113341CF2271FCC7DC3BD13DBCC7DD0BD6501F67B
S113342C965A4F3406CC000E3406CC0014BD128EC2
S113343C3264F6965AC1421027003DC1431027004E
S113344C40C1442721C1462714C1532707C15A2719
S113345C1E160034BD349AF7965A16FFB1BD356D5D
S113346CF7965A16FFA8BD3714F7965A16FF9FBD48
S113347C3854F7965A16FF96BD3981F7965A16FFAB
S113348C8DBD166BCC000139BD166B5F4F39327E86
S113349CF696587C9658F195902505C6414F359073
S11334AC306134108E95911F10BD14853262CC009E
S11234BC0134068E95913410E6654F3406F6966A
S11334CB593406CC0053BD16C33268CC0001340604
S11334DB8E95F434103064341030671F10BD19CC42
S11334EB3266108300001027006D108300451027EF
S11334FB004E1083004E2711108300541027004DEB
S113350B108300592709160054F6965A4F3590E646
S113351BE4F196592706F6965A4F3590E6614F34E7
S113352B068E95F41F10BD14FA32627F9658F696E8
S113353B59CB018640BD4541F79659C6464F359048
S113354B8E95F41F10BD0E2AC6414F3590F6965733
S113355B2705C6414F3590F6965A4F3590C6414FC5
S113356B359032E8CCF696587C9658F19590250711
S113357BC6414F32E834397F9657FC950B1083FFC5
S113358BFF10260074FC9665C30030E762C62EE775
S113359B63FC968F340630661F10BD65FB3262F6F2
S11335AB94F32713CC7DDD340630641F10BD510A10
S11235BB3262FD950B2011CC7DE0340630641F85
S11335CA10BD510A3262FD950BFC950B1083FFFF67
S11335DA262830623410CC7DE23406CC0005BD0DB9
S11335EA6F32645F4FBD3D59ED7E2607C6434F32A5
S11335FAE83439C6534F32E83439CC7DE53406CC45
S113360A000234065F4FBD126A326430623410CC51
S113361A00023406CC0014BD126A3264CC7DEFBDBC
S113362A6501FC968FBD6617E761F694C74F3406A9
S113363AFC968F3406E6654F3406F696593406CC62
S113364A0046BD16C33268F694C74F34068E95F405
S113365A34103064341030671F10BD19CC32661030
S113366A83000010270094108300451027006C1073
S113367A83004E2711108300541027006D10830015
S113368A59272016007D6AE4E6E4C1002404C63FF3
S113369A2002E6E4E7E4F196592708F6965A4F32EF
S11336AAE83439E6E4F196592708F6965A4F32E88F
S11236BA34397F9658F69659CB018640BD454169
S11336C9F79659CC000134068E95911F10BD1DEC57
S11336D93262FD965BC6444F32E834398E95F41F45
S11336E910BD0E2AC6414F32E83439F69657270CD5
S11336F95F4FBD0D6FC6414F32E83439F6965A4FC4
S113370932E83439C6414F32E83439327DF69658B5
S11337197C9658F195902506C6414F326339F69443
S1133729C74F34068E95913410FC965B4F3406F6D8
S113373996593406CC0044BD16C33268F694C74F73
S113374934068E95F434103064341030671F10BD7C
S113375919CC326610830000102700E2108300455B
S1133769102700BC1083004E271110830054102722
S113377900BC10830059271F1600CA6AE4E6E4C195
S1133789002404C63F2002E6E4E7E4F1965927073A
S1133799F6965A4F326339E6E4F196592707F696B5
S11337A95A4F3263397F9658F69659CB018640BDF4
S11237B94541F796595F4F34068E95911F10BD09
S11337C81DEC3262FD965B1083FFFF2606C65A4F36
S11337D8326339F695F4E762E661C101261AE662B6
S11337E8C15A26037F9694E662C1582704C15A2613
S11337F807E662CBC0F79657F696574F1083001822
S1133808270AF696574F1083001A260FCC7DF0BD71
S11338186501BD125EC65A4F326339C6444F3263DE
S1133828398E95F41F10BD0E2AC6414F326339F6FE
S11338389657270B5F4FBD0D6FC6414F326339F65C
S1133848965A4F326339C6414F326339327DF69600
S1133858587C9658F195902506C6414F3263396FC6
S113386862F696574F10830018270AF696574F109A
S113387883001A2609C644F79591C601E762F694AF
S1133888C74F34068E95913410E6664F3406F69683
S1133898593406CC005ABD16C33268F694C74F345F
S11338A8068E95F434103064341030671F10BD1937
S11238B8CC326610830000102700B11083004546
S11338C71027008B1083004E2711108300541027F4
S11338D7008B10830059271F1600996AE4E6E4C198
S11338E7002404C63F2002E6E4E7E4F196592707DB
S11338F7F6965A4F326339E6E4F196592707F69656
S11339075A4F3263397F9658F69659CB018640BD94
S11339174541F79659FC950BBD4B8FCCFFFFFD95A1
S11339270B5F4FBD3D59ED7E2606C6424F326339C4
S1133937F696574F1083001A260F5F4FBD3D59ED7A
S11339477E26F7C6424F326339C6464F3263398EF5
S113395795F41F10BD0E2AC6414F326339F69657A8
S1133967270B5F4FBD0D6FC6414F326339F6965A29
S11339774F326339C6414F326339327EF696587CEB
S11339879658F195902505C6414F3590F694C74F43
S113399734068E959134105F4F3406F696594F349A
S11339A706CC0042BD16C33268F694C74F34068E60
S11239B795F434103064341030671F10BD19CCF0
S11339C63266108300001027007810830045102704
S11339D600541083004E27111083005410270053FF
S11339E610830059271E16005F6AE4E6E4C100242A
S11339F604C63F2002E6E4E7E4F196592706F69664
S1133A065A4F3590E6E4F196592706F6965A4F35FD
S1133A16907F9658F69659CB018640BD4541F79658
S1133A2659C6434F35908E95F41F10BD0E2AC641D4
S1133A364F3590F69657270A5F4FBD0D6FC6414F17
S1133A463590F6965A4F3590C6414F359034063226
S1133A567EE6672603BD3D58EC62FD9660BD3AA836
S1133A66ED7E26055F4F326439C603E7F8028E6D94
S1133A7645AFE4AEE4EC81AFE410B395582709EC06
S1133A86E4C30002EDE420EBF694C258584FAEE4CA
S1133A96AA84EA01E7F802EC62BD3CFFCC000132DD
S1133AA664393406327BE6F805E762AE65E601E77B
S1123AB663E603E7647F96626F035F4FEDE4AE50
S1133AC565E603271DC603E7F8055F4FEDE4E6F851
S1133AD505C4F3C100260BC601F79663CC00013279
S1133AE56739E662E7F805E663AE65E701E664AEC5
S1133AF565E703C601F796625F4F326739F694F0BE
S1133B052706FC92B5FD9507C601F76D515F4F3445
S1133B1506FC9507BD3A5332627F965739F694F001
S1133B252706CCFFFFFD95077F6D515F4F3406FCDB
S1133B359507BD3A533262F696572706CC7E07BDE4
S1133B456501393406327A5F4FEDE4EC6C10A3E479
S1133B55102F0045FC94CBFE94C9ED64EF62EC662E
S1133B65BD3CA2ED7E26173062BD5869BD5849009B
S1133B7500000026E9BD3C02CC0001326839EC6A3C
S1133B85AEE4308B3410EC68BD3CABE7F1F7965FDF
S1133B956C6126026CE416FFB2F696912605F6943E
S1133BA5F1270BEC6CBD658F8E94DDBD581D5F4F01
S1123BB53268393406327EEC682607EC66BD664A
S1133BC417ED685F4FEDE4EC6810A3E42F18EC6282
S1133BD43406EC68AE62E68B4FBD3CC932626C615C
S1133BE426026CE420E1F696912605F694F1270B5F
S1133BF4EC68BD658F8E94E1BD581D326439327F03
S1133C04F692AC10260092F696641026008BFC9271
S1133C14B5BD3CA2ED7E270AFC92B5BD3CABE7E4FE
S1133C24200EF694F02707F6965FE7E420026FE48B
S1133C34E6E4C47FE7E47F965F4F10830018270906
S1133C44E6E44F1083001A2609E6E4F796574F3248
S1133C546139E6E44F108300042626F694F227170C
S1133C647F94F2FC950F1083FFFF2710BD4B8FCC7C
S1133C74FFFFFD950F2005C601F794F2BD128D20B8
S1133C8418E6E4F192AE2611FC9507BD3CAB840022
S1133C94C47FE7E4F192AD26EF5F4F326139340615
S1133CA4E6F4C4014F35903406ECE4BD3CA2ED7E49
S1123CB427F7AEE4E6014F35903406BD3C02E637
S1133CC3F4C4024F35903404327CFC94CBFE94C983
S1133CD3ED62EFE4EC67BD3CBDED7E261630E4BD3A
S1133CE35869BD58490000000026E9F6965727E4B1
S1133CF3326539E664AE67E7013265393406ECE4CC
S1133D03BD3CA2ED7E2707ECE4BD3CAB20F035902F
S1133D133406C660E7F4CC012CBD3D2B5F4F34065B
S1133D23EC62BD3A533264393406327CEC642722A4
S1133D33BD5728BD4C51447A0000BD4FF04649900D
S1133D4300BD4F21ED62EFE430E4BD5869BD66B7B1
S1133D5326F6326639393404327EE6622712C60106
S1133D63F79693F69692CBFFF79694C601F77E7C6B
S1133D73F69691C102271CF67E7C4F3406F6969381
S1133D83584F8E9667EC8BBD3DF43262EDE47F7E33
S1133D937C201BF696937C9693584F8E9667EC8BF8
S1133DA3EDE4F696947A9694C1001027003EECE471
S1123DB31083FFFF2608CC7E09BD0D47202EECA0
S1133DC2E42718ECE4FD968FF69691C1022706FCCF
S1133DD2968FBD124ECC00013263397C9693C60194
S1133DE2F77E7C7A9694F696941026FF845F4F327F
S1133DF263393406E6652713ECE4BD3FE1FD7E7DBD
S1133E021083FFFF2605CCFFFF35908E7E7F341092
S1133E12FC7E7DBD40BA32621083FFFF2719ECE4B9
S1133E2234068E7E7F1F10BD3E433262ED7E27DB59
S1133E328E7E7F1F103590FC7E7DBD5B2F5F4F35DC
S1133E4290340632E9FEF8ECE9010834063068AF32
S1133E52641F10BD65FB3262EC62BD124EECE901D7
S1133E620C340630E9008AAFE900881F10BD65FBF7
S1133E723262ECE90086BD124EE6F9008610270094
S1133E8288E6F90086C12A10260047EC62ED64AE8A
S1133E92E900863001AFE90086E6845D2608CC009D
S1133EA20132E9010A39E6F802271AECE9008634FC
S1123EB206EC64BD3E433262ED7E2609EC62C32A
S1133EC10001ED6220E1E6F8021026FFADEC64ED9D
S1133ED1622026ECE900863406E6F8044FBD3F1A59
S1133EE13262EDE4ED7E26075F4F32E9010A39ECD7
S1133EF1E90086E3E4EDE90086E6F8021027FF7A9B
S1133F01EC62C30001ED6216FF70E6F80226035C61
S1133F1120015F4F32E9010A393404327BEC68ED48
S1133F21631F01E684E7E4C13F10260006E665103D
S1133F312600A7E6E4C15B102600806F625FE7619B
S1133F41AE633001AF63E684C15E260BC601E7624E
S1133F51EC63C30001ED63E6F803E7E45D102700B9
S1133F6145C15D1027003FE6F803C12D262EAE633F
S1133F71E61FE1652226E601E1652520E61FE10150
S1133F81221AAE63E601E7E45D270DC15D27091F2F
S1133F9110C30001ED6320EAC601E761EC63C300CD
S1133FA101ED6316FFB1E661E16226055F4F3266FA
S1123FB139EC63A368C30001326639E6E4C15EEC
S1133FC0260EAE63E601E1652706CC0002326639AF
S1133FD0E665E1E427055F4F326639CC00013266BD
S1133FE0393406327CF6CC0C4FFD9665EC64BD6624
S1133FF017ED62108300012617E6F8044FBD57C57C
S1134000ED7E270CE6F804CBD04FFD966516006ACA
S1134010E6F8044FBD57C5ED7E2721AE64E601C125
S11340202E2619E6F804CBD04FFD96651F10C30069
S11340300234061F10BD65FB3262203EEC64E3626D
S11340408EFFFF308BE6844FBD57C5ED7E272BECEA
S113405064E3628EFFFE308BE684C12E261CEC6482
S1134060E3628EFFFF308BE684CBD04FFD9665EC88
S113407064E3628EFFFE308B6F84CC0144BD5A77BB
S1134080EDE4108300002606CCFFFF326639FC966F
S113409065AEE4E703C606E7F45F4F3406EC62BDA1
S11340A04FCE32621083FFFF260BECE4BD5B2FCCB6
S11240B0FFFF326639ECE43266393406327CC6DF
S1137D4474696E67206E6577206E616D6500000A44
S1137D5400257300526563656976696E673A20008D
S1137D64004E65772066696C65206E616D653A2006
S1137D7425730A002564005472616E73666572206B
S1137D8461626F727465642E0A0046696C6573706F
S1137D946563287329207265717569726564004E80
S1137DA46F2066696C65732073656C6563746564C0
S1137DB40053656E64206661696C65642E0000532B
S1137DC4656E642073746174653A200053656E644F
S1137DD42073746174653A20006272007200257322
S1137DE40053656E64696E673A2000005472616ED4
S1137DF47366657220696E746572727570746564F5
S1137E042E0A000A004572726F72206F70656E69E3
S1137E146E67206469726563746F7279002E004B17
S1137E2445524D49542E484C500072004E6F206800
S1127E34656C7020617661696C61626C652E000B
S11340BF07E7F8045F4F3406EC66BD4FCE3262104B
S11340CF83FFFF102700A05F4FEDE4ECE4108300A3
S11340DF082C1BAE68308B3410EC66E3628E000440
S11340EF308BE684E7F16C6126026CE420DDAE6868
S11340FF6F08E6F8082606CCFFFF326639E6F808A3
S113410FC1FF1027FFAECC7E213406EC6ABD65BC1F
S113411F3262EC68BD6617ED625F4FEDE4ECE410BC
S113412F8300032C1DE362AE68308B3410EC66E31E
S113413F628E000C308BE684E7F16C6126026CE42E
S113414F20DBEC68E3628E0003308B6F84AE64EC8B
S113415F8815FD9699CC0000CE0000FD9697FF962A
S113416F95CC0001326639CCFFFF32663932E9FF54
S113417F6FF6CC0CE7E90083F6969BF7CC0CCC7E5C
S113418F2E3406CC7E23BD510A3262EDE41083FF38
S113419FFF260BCC7E30BD0D4732E9009139F696E0
S11241AF92C101262330623410EC62BD430C32FE
S11341BE62ED7E2706E662C13026EB30623410ECE7
S11341CE62BD433832621601246FE900865FE7E967
S11341DE0085E7E90084E6E90086102600F6E6E9A4
S11341EE0084102600EE30623410EC62BD430C32B3
S11341FE62ED7E102700DDCC0001EDE90087F69616
S113420E924F10A3E900872FCDECE9008758498E11
S113421E9667EC8BBD0D1B30621F10BD0D1B3062FB
S113422E1F10BD6617C3FFFEEDE9008BECE9008796
S113423E58498E9667EC8BBD6617EDE9008D10A379
S113424EE9008B2C022004ECE9008BEDE9008F30A1
S113425E621F10BD44C8EDE90089E6E90085271404
S113426EECE9008910A3E900872C09C601E7E900EF
S113427E8616FF62ECE9008710A3E900892640EC5C
S113428EE9008F3406ECE9008958498E9667EC8B69
S113429E340630671F10BD66333264108300002667
S11242AE1EC601E7E90085F69692CBFF4F10A3D9
S11342BDE900871026FF20C601E7E9008416FF17E1
S11342CDE6E900851027FF0F6CE9008826046CE9E8
S11342DD008716FF2AE6E90084270D30623410ECBE
S11342ED62BD433832622006CC7E43BD0D47ECE4FB
S11342FDBD4B8FE6E90083F7CC0C32E900913934DC
S113430D06ECE43406CC00803406EC68BD696132F9
S113431D64108300002710E6F8044FBD57C5ED7EE9
S113432D27DFCC000135905F4F3590340632E9FF1D
S113433D7FECE90085C300013406CC7E51BD632EAC
S113434D3262ECE900813406CC0080340630641FFF
S113435D10BD69613264108300002713E6E44FBD7C
S113436D57C5ED7E260930E41F10BD650120D3CC61
S113437D7E56BD650132E900833934063274E6F8A0
S113438D0C4FBD57EFED7E2709EC6CC30001ED6CAE
S113439D20ECCC0001ED68E6F80CC12B2609EC6C81
S11243ADC30001ED6C2013E6F80CC12D260CECB7
S11343BC6CC30001ED6CCCFFFFED68CC0000CE00AB
S11343CC00ED62EFE4E6F80C4FBD57C5ED7E2727F0
S11343DCEC62EEE4BD4FF04120000034063440E6BC
S11343ECF810CBD0BD5738BD49D8ED62EFE4EC6C76
S11343FCC30001ED6C20CEE6F80CC12E2607EC6C44
S113440CC30001ED6CCC0000CE3F80ED66EF64E69A
S113441CF80C4FBD57C5ED7E2736EC62EEE4BD4F6C
S113442CF04120000034063440E6F810CBD0BD57E0
S113443C38BD49D8ED62EFE4EC66EE64BD4FF04153
S113444C200000ED66EF64EC6CC30001ED6C20BF42
S113445CE6F80C4FBD6675108300651026004BEC16
S113446C6CC30001ED6CBD44C8ED6AEC6A108300AA
S113447C002C17EC62EEE4BD4C5141200000ED62BF
S113448CEFE46C6B26026C6A20E1EC6A108300008A
S113449C2F18EC62EEE4BD4FF041200000ED62EF0A
S11244ACE4EC6A830001ED6A20E0EC68BD572858
S11344BB30E4BD4FF83064BD4C59326E393406329A
S11344CB7CE6F804C1092704C1202609EC64C30067
S11344DB01ED6420ECCC0001ED62E6F804C12B275E
S11344EB04C12D2614AE64E680AF64C12D2605CC21
S11344FBFFFF2003CC0001ED625F4FEDE4E6F8040F
S113450B4FBD57C5ED7E2722ECE434065849584974
S113451BE3E158493406E6F8064FE3E1C3FFD0ED77
S113452BE4EC64C30001ED6420D3EC623406EC626A
S113453BBD56E53266391A0120021CFE34014D26A4
S113454B063501C6FF4F39A7E26FE26CE46D612BB0
S113455B0668616CE420F64FE0612406EB611CFEF7
S113456B20021A014964616AE426ED3262350125A1
S113457B021F894F393406327C5F4FEDE430E4344B
S113458B10EC6A3406EC68BD000032645F4FBD4921
S113459BBF326639AE628D7B3401AF6335012002C5
S11245AB1CF71A0134018E000035012014AE6292
S11345BA8D623401AF638E7FFF350120058EFFFFC4
S11345CA1CF6327D3401ED62260635011F10203EA9
S11345DA8601A7616D622B08686369626C6120F4C5
S11345EAEC666F666F67A3622406E3621CFE200210
S11345FA1A0169676966646266636A6126E8350155
S113460A25063401EC6635012A0440508200AE6363
S113461A32676E8434401F033410A8E11CFE34014F
S113462A1F108D081F011F308D0235C14D2A044009
S113463A5082003934063440CC00013406EC6C3420
S113464A06EC6C3406EC6C3406EC6AEE68BD467B08
S113465A326C39340634405F4F3406EC6C3406EC61
S113466A6C3406EC6C3406EC6AEE68BD467B326C3C
S113467A393406344032E8EB306E3410ECE819EE83
S113468AE817BD67D43262EC6F10837FFF102600EF
S113469A98E66E2705CC000120025F4FEDF81F5FF4
S11246AA4FEDF81DECE813EEE811BD5849000080
S11346B900002618CC7E5834068E7EB11F10BD65C5
S11346C9FB32628E7EB11F1032E81939CC7E5C341C
S11346D9068E7EB11F10BD65FB3262CE7EB1E64403
S11346E9EBE811E744E6E812545454544FBD493AEF
S11346F98E7EB1E707E6E812C40F4FBD493A8E7EB4
S1134709B1E708E6E813545454544FBD493A8E7E30
S1134719B1E709E6E813C40F4FBD493A8E7EB1E704
S11347290A8E7EB11F1032E81939ECE81B10830098
S1134739002C055F4FEDE81BECE81B1083004F2D9F
S113474906CC004EEDE81B5F4FED6CEDF81F8E7E35
S1134759B1AF68ECE817EEE815BD4BE500000000C1
S11347692C15CC0001EDF81FECE817EEE815BD5146
S113477903EDE817EFE81530E43410ECE819EEE836
S113478917BD49503262EDE817EFE8158E7EB11F67
S113479910C30050ED6AEC62EEE4BD4BE500000085
S11247A90010270062EC62EEE4BD4BE500000057
S11347B800273A30E43410EC64EE62BD4C514120D9
S11347C80000BD49503262ED66EF64BD49E23CF534
S11347D8C28FBD4FF041200000BD4F96C30030AEDC
S11347E86AE782AF6A6C6D26026C6C20B98E7EB162
S11347F81F10C3005010A36A234AAE6AE680AF6A4A
S1134808AE68E780AF6820E5ECE817EEE815BD4B25
S1134818E5000000002F2DECE817EEE815BD4FF079
S113482841200000ED66EF64BD4BE53F8000002C9D
S113483813EC66EE64EDE817EFE815EC6C83000101
S1134848ED6C20D3ECE81BC37EB1ED6AE6E82226C2
S113485806EC6AE36CED6AEC6CEDF81DEC6A108307
S11348687EB1240C7F7EB18E7EB11F1032E81939D7
S1134878EC6810A36A22408E7EB11F10C30050104A
S1134888A3682333CC0000CE412030E815BD4FDFA8
S113489830643410ECE819EEE817BD49503262ED83
S11248A8E817EFE815EC66EE64BD4F96C30030D9
S11348B7AE68E780AF6820B98E7EB11F10C3005081
S11348C710A36A240C6F884F8E7EB11F1032E8192B
S11348D739EC6AED68E6F80ACB05E7F80AE6F80A60
S11348E7C13910230041C630E7F80AEC6A10837E09
S11348F7B1230A1F01301FAF6A6C8420E0C631E779
S1134907F80AECF81DC30001EDF81DE6E82226CDF0
S1134917EC6810837EB12305C630E7F808EC68C35A
S11349270001ED6816FFB66FF8088E7EB11F1032CE
S1134937E819393404E6E4CB30E7E4C1392304CB7E
S1134947072002E6E44F326139340634403278EC0A
S11349576AEE68BD4F21ED66EF64BD58497FFFFFDE
S1134967FF270DEC66EE64BD58498000000026134E
S1134977EC6AEE68AE6EED02EF84CC0000CE000068
S1134987326C39EC66EE64BD5760AE6EED02EF84AF
S1134997EC6AEE68AE6EBD4A11ED62EFE4BD4BE51D
S11249A7000000002C0BEC62EEE4BD5103ED6246
S11349B6EFE4EC62EEE4326C393406ECE4BD49C84B
S11349C635903406ECE4BD695E35908D51ED02EF09
S11349D6843930628D48AEE432666E84AEE48D3E30
S11349E635106E0434163440EC02EE8430E48D1B2C
S11349F632643510ED02EF843930628D0EAEE43246
S1134A06666E84AEE48D0435106E043410171DCC26
S1134A163401EC8488801F03EC023501200D341028
S1134A26171DB93401EC02EE8435012B0F2512272C
S1134A3634171DA82B282526270E8D3E171E17353D
S1134A4690171D982B182504326720F0A6E4A16759
S1134A56326727E88604A763EC69ED6420DE171D38
S1134A66F532673590171D742BF425F226F0A6E46B
S1134A76A167326727C66FE420C26FE26FE2306C2B
S1134A86EE6511A38427302E153341646766686684
S1134A9669666AE661562402CA01E76120E46C018C
S1124AA626026C846402660366046605E6E45621
S1134AB52402CA01E7E420CBA66BA164263CE6E404
S1134AC5EB61E7E4EC04E96AA969ED04EC02E96841
S1134AD5A967ED02241C6602660366046605E6E41E
S1134AE55624028A01E7E4EC84C30001ED8410290D
S1134AF50087E6E4EE62326B6EC430023367ECE4A1
S1134B056D6B27041E311E896F6BE7E2A0E0A7E4F5
S1134B15EC02E243A242EDE810EC84E241A2C4EDCA
S1134B256E24278680A76B636E636F63E81063E862
S1134B3511A6E4438B01A7E4ECE810C9008900ED54
S1134B45E810EC6EC9008900ED6E6DE42610EC6E7C
S1134B55260CECE8102607CC8000ED6C20946D6ED5
S1134B652B90EC6C8300012989ED6C68E469E811EC
S1134B7569E810696F696E20E5CC7FFFED6C4F5FC6
S1134B85A7E4ED6EEDE81016FF683406ECE483FF48
S1134B95FF10830004221B8E4BA358496E9B4BAD1B
S1124BA54BAD4BB24BB24BB2CCFFFF3590CC00B3
S1134BB4013590C604E7F45F4F3406EC62BD4FCE72
S1134BC432621083FFFF2605CCFFFF3590ECE4BD71
S1134BD45B2FCC0001359030628D0C351032646E3D
S1134BE48435108D026E0434101E034D2A028D2C5C
S1134BF43446EE02EC842A028D22AEE4EDE4EC6247
S1134C04EF62A36234011F10E2621FA9E4E0CAFB4D
S1134C14A2E43401E4E01F9A32643590888043535B
S1134C241E304353C30001240233411E3039341669
S1134C343440EC02EE8430E48D1B32643510ED0212
S1134C44EF843930628D0EAEE432666E84AEE48D48
S1134C540435106E043410171B842B1325162743B4
S1134C64EC02EE84171B772B20254D27588D5B17F8
S1134C741BE63590EC02EE84171B632B0C2518A657
S1134C8467A8E4A767326720E6171BCC3267359020
S1134C94CC7FFFED686C6A32676C636FE4EC69ED9A
S1124CA46420CCEC02EE84171B3427E42BDBA630
S1134CB367A8E4A767326720B7CC8000ED61A667D5
S1134CC3A8E4A7E420C4CC7FFF20F14F5FEDE3ED1C
S1134CD3E3A666A86DA76DEC6EA3672807102500ED
S1134CE39516008D830001ED6EAE69EE6BACE81092
S1134CF3222B260611A3E8122223EC6EC30001ED36
S1134D036E10837FFF276A64E81066E81166E81271
S1134D1366E81366E466616662666320D08621A74B
S1134D236630E8106A66273A68636962696169E410
S1134D3369036902690169842516EC02A36B1F03E5
S1134D43EC84E26AA26925DCEF02ED846C6320D46F
S1134D53EC02A36BED02EC84E26AA269ED846C635A
S1134D6320C2EC62ED02ECE4ED84EE64326D5F6E1E
S1134D73C4CC7FFF2003CC8000ED6E4F5FEDE810C1
S1134D83EDE81220E53406327E6FE4F6CC0CAE6611
S1134D93E703E6F8024FBD57C5ED7E271CAE62E676
S1124DA380AF62CBD0AE66E703AE62E680AF624C
S1134DB2C12E2706CCFFFF326439E6F8024FBD57F5
S1134DC2A9ED7E2606CCFFFF3264396F61E6F80254
S1134DD22738C12E27344FBD4EF8ED7E271DE661DC
S1134DE2C108241DEC66C300043406E6636C634FF9
S1134DF2E3E13406E6F804E7F12006CCFFFF32646F
S1134E0239EC62C30001ED6220C3E661C108240EDD
S1134E124FE3668E0004308B6F846C6120EC6F610B
S1134E22E6F802C12E10260056AE62E6014FBD57C7
S1134E32A9ED7E10270048EC62C30001ED62E6F89A
S1134E42022738C12E27344FBD4EF8ED7E271DE6CA
S1134E5261C103241DEC66C3000C3406E6636C6373
S1134E624FE3E13406E6F804E7F12006CCFFFF3213
S1134E726439EC62C30001ED6220C3C601E7E4E6D3
S1134E8261C103240E4FE3668E000C308B6F846C79
S1134E926120ECE6F802C12E2621AE62E6014FBD86
S1124EA257C5ED7E2715AE623001AF62E684CBB3
S1134EB1D0AE66E703EC62C30001ED62E6F802C11D
S1134EC12E2607EC62C30001ED62E6F8022706CC48
S1134ED1FFFF326439E6E42618E669C10B2306CCE8
S1134EE1FFFF326439E6694F3406EC68BD658832E8
S1134EF162CC00013264393404E6E44FBD57A9EDB4
S1134F017E2617E6E44FBD57C5ED7E260DE6E4C1C6
S1134F115F2707C12D27035F2002C6014F32613984
S1134F2134108D52A661817F27376F61811727184D
S1134F312D0D68646963696269612B254A20ED4C12
S1134F4164626663666420E4A6E03546270F435332
S1134F511E034353C300012406334120021E0335BB
S1134F61906DE432652707CE80004F5F3590CE7F88
S1134F71FFCCFFFF3590327D1E036FE4584966E490
S1134F81807FA7615481812F02CA80E7621F30EEBE
S1134F9163ED636EC417FF88118300002E052D078E
S1124FA14D2A03CC7FFF391183FFFF26034D2BCD
S1134FB0F6CC80003917FF691183000027E92D041E
S1134FC0CCFFFF394F5F398DEC4D27DB20F21F01F9
S1134FD0A663BDD40626041F894F39CCFFFF398D43
S1134FE017ED02EF843930628D0EAEE432666E84C2
S1134FF0AEE48D0435106E0434101717E52B132519
S1135000162741EC02EE841717D82B20254B27498D
S11350108D4F1718473590EC02EE841717C42B0CEC
S11350202716A667A8E4A767326720E617182D326B
S1135030673590CC7FFFED6832678603A763EC6920
S1135040ED6420CEEC02EE841717972BDF25E4A63F
S1135050E4A867A767326720B9A6E4A867A7E42095
S1135060CB4F5FEDE3EDE3A666A86DA76DEC6EE3B1
S1135070672804257F2078C3000110837FFF276FF2
S1135080ED6E30E8108620A7664FA6038401270E34
S1135090EC62E36BED62ECE4E96AA969EDE466E4D1
S11250A066616662666366846601660266036A19
S11350AF6626D76DE42B1BEC6E830001ED6E29355C
S11350BF680369026901698469636962696169E402
S11350CF2AE5E6846D0126086D0226046D03270286
S11350DFCA01EEE4EF84EE62EF02EE64326D6EC449
S11350EFCC7FFF2003CC8000ED6E4F5FEDE810ED19
S11350FFE81220E61E3088801E30393406327C6F69
S113510F63C601E762E6F8082730AE68E680AF6849
S113511F4FBD667510830062271A1083007227082B
S113512F10830077270820DDC601E76220D7C60267
S113513FE76220D1C601E76320CBE662C1022605F0
S113514FEC64BD66C6CC0144BD5A77EDE410830010
S113515F002606CCFFFF326639E66327045F4F2033
S113516F03CC00013406EC623406EC68BD4D883282
S113517F641083FFFF260BECE4BD5B2FCCFFFF32E3
S113518F6639E662E7F45F4F3406EC62BD4FCE3208
S112519F621083FFFF260BECE4BD5B2FCCFFFFF8
S11351AE326639E6632707C6FFAEE4E7883BCCFFD9
S11351BEFFAEE4ED8901405F4FAEE4ED890142ECB0
S11351CEE4326639340632E9FF0030E90106341060
S11351DEECE90106340630641F10BD5BF83264EC52
S11351EEE90100340630621F10BD51FF32E901049B
S11351FE393406327DEC67108300022608EC63BD59
S113520E6501326539EC63ED61AE61E680AF61E74D
S113521EE45D2718EC673406E6624FBD63643262C0
S113522E1083FFFF26E3CCFFFF326539EC63326552
S113523E39CC0001BD525E393406ECE41083FFFF15
S113524E2607C61AF77F013590E661F77F01359080
S113525E3406327D6F62EC63108300011026004920
S113526EF67F012719F67F014FEDE47F7F0110834E
S113527E001A2605CCFFFF2002ECE4326539F6CC89
S113528E232610F6CC26270BC601E762FCCC26EDAE
S112529E632016BD5316EDE41083001A2606CCC8
S11352ADFFFF326539ECE4326539AE63E602C102C3
S11352BD260AC612E701CCFFFF326539E662261EC7
S11352CDAE63EC8901401083FFFF2712EC89014086
S11352DDEDE4CCFFFFED890140ECE43265396FF864
S11352ED035F4F3406EC65BD4FCE3262EDE4AE6321
S11352FDE6883BC1FF270DECE41083000D2605CC99
S113530D000AEDE4ECE4326539BDCD151F894F3942
S113531D340632E8EA5F4FED64AEE81AE680AFE892
S113532D1AE7615D1027033CE6F8162606EC643295
S113533DE81839E6614FBD57EFED7E26DCE661C115
S113534D25271E30E8161F10BD5677E1612706ECA0
S113535D6432E81839ECE816C30001EDE81616FFBF
S113536DB86F66C601E7E4CC0100ED6BE6F81AC12F
S113537D2A260BECE81AC30001EDE81A6FE4E6F8EF
S113538D1A4FBD57C55D270A30E81A1F10BD5BBE05
S112539DED6BAEE81AE680AFE81AE7614FBD6624
S11353AC75C16C2610C601E76DAEE81AE680AFE84D
S11353BC1AE76120026F6DE6614FBD6675C063C16B
S11353CC15102202524F8E53D958496E9B55F854DE
S11353DCFF56235405562354FF562356235623565F
S11353EC235623562354F8562356235623559D5699
S11353FC2355185623562354F1ECE816ED693069FD
S113540C1F10BD5677E761C12B2704C12D2607EC6D
S113541C69C30001ED69E6F8094FBD57C55D27095D
S113542CEC69C30001ED6920EDE6F809C12E261ADA
S113543CEC69C30001ED69E6F8094FBD57C55D275A
S113544C09EC69C30001ED6920EDE6F8094FBD666E
S113545C75C165262CEC69C30001ED69E6F809C138
S113546C2D2704C12B2607EC69C30001ED69E6F86E
S113547C094FBD57C55D2709EC69C30001ED6920CF
S113548CEDECE81610A3692606EC6432E81839EC46
S112549C69A3E81610A36B2F07ECE816E36BED7A
S11354AB69E6F809E7616FF809E6E4270CECE816FE
S11354BBBD4387EDE814EFE812EC69EDE816E661FD
S11354CBE7F809E6E41027FE52ECE814EEE812AE16
S11354DBE81C3002AFE81CAE1EED02EF846C6526AF
S11354EB026C6416FE35CC0010ED622025CC00084E
S11354FBED62201E30E8161F10BD5677C12D260D08
S113550BC601E766ECE816C30001EDE816CC000A09
S113551BED62CC0000CE0000EDE810EF6EEC6234CF
S113552B0630E8181F10BD56774FBD56A4326210D3
S113553B83FFFF2606EC6432E81839EC623406E686
S113554BF8184FBD56A43262ED671083FFFF102786
S113555B00CCEC6B830001ED6BC30001ED7E1027D7
S113556B00BCEC67BD658F34063440EC66BD658FBB
S113557B34063440ECE818EEE816BD59F13264BD3C
S113558B5824EDE810EF6EECE816C30001EDE816B5
S112559B20A930E8161F10BD5677ECF81CED69F7
S11355AAEC6B830001ED6BC30001ED7E2725E6F861
S11355BA1627204FBD57EFED7E2618E6E42709E6A5
S11355CAF816AE69E780AF69ECE816C30001EDE8A6
S11355DA1620CDE6E41027FD436C6526026C646F41
S11355EAF809ECE81CC30002EDE81C16FD2EEC6B6E
S11355FA1027FD28E6E42715E6F816AEE81C300263
S113560AAFE81CAE1EE7846C6526026C64ECE816EF
S113561AC30001EDE81616FD03EC6432E81839E616
S113562AE41027FCF7E666270DECE810EE6EBD5A87
S113563A67EDE810EF6EE66D2715ECE810EE6EAE36
S113564AE81C3002AFE81CAE1EED02EF84200FEC1A
S113565AE810AEE81C3002AFE81CAE1EED846C659F
S113566A26026C6416FCB5EC6432E8183934063246
S113567A7FAEF801E684E7E4E6E44FBD57EFED7E3A
S113568A2712ECF801C30001EDF801AEF801E68433
S112569AE7E420E4E6E44F3263393404E6E44FF6
S11356A9BD6690E7E4C141250AC15A2206CBC9E780
S11356B9E42017E6E44FBD57C55D2708E6E4C0308A
S11356C9E7E42006CCFFFF326139E6E4E16425060C
S11356D9CCFFFF326139E6E44F326139327B6FE442
S11356E98D33ED61EC678D2DED67A662E6683DEDBE
S11356F963A661E6683D1F985FE363ED63A662E60E
S1135709673D1F985FE3636DE42A0440508200AE4D
S11357196532696E844D2A06636240508200394DB0
S11357292A0E405082008D081E038A801E03394FB9
S1135739ED7E271D6FE24D2B0658496CE420F734A2
S11357490448C68EE0616F6135401E8944561E03C4
S113575939CE00004F5F393410118300002604ED5F
S11357697E273B32796FE41E034D2A131A0166E43E
S113577943531E034353C30001240233411E03ED63
S113578963EF65CC001FED616D632B0F6866696576
S112579969646963830001ED6120ED1710B53574
S11357A8903406ECE4BD5808ED7E260CECE4BD57B5
S11357B8DAED7E26035F2002C6014F35903404E6F5
S11357C8E4C1302508C1392204C60120015F4F32E3
S11357D861393404E6E4C1612508C17A2204C601AA
S11357E820015F4F3261393404E6E4C120270BC13C
S11357F80A2707C10927035F2002C6014F3261390E
S11358083404E6E4C1412508C15A2204C601200132
S11358185F4F3261398D15ED02EF843930628D0C9A
S1135828351032646E8435108D026E04E3021E0353
S1135838E901A9841E033930628D0C351032646E77
S11358488435108D026E043446A30234011F30E2FD
S1135858011FA9E4E0CAFBA2843401E4E01F9A35DD
S1135868C6EE84EC028300012402335FEF84ED0268
S113587839341034063440EC02EE8430E48D40327E
S1135888643510ED02EF8439341034063440EC02E8
S1125898EE8430E48D7232643510ED02EF843902
S11358A730628D1C351032646E8430628D5B351026
S11358B732646E8435108D086E0435108D4B6E047A
S11358C734101E033446A884EE02AE843450327C6E
S11358D7A7E230698D1930658D153061170084A6EC
S11358E7E02A0430688D0C326835461E0335906D06
S11358F7842A15EC8443531F03EC024353C300016A
S1135907ED0224023341EF843934101E033446EE8A
S113591702AE843450327CA7E230698DD230658D73
S1135927CE30618D3EA6E02A0430E48DC635461E8E
S113593703326835901E033446EC66EE683446320B
S11359477C30E48D1E326835461E03391E03344607
S1135957EC66EE683446327C30E48D0735461E0328
S11359673268394F5FED84ED028621A7E26AE427A6
S113597726680B690A690969086903690269016983
S113598784EC02A3061F03EC84E205A20425DEEFE0
S112599702ED846C0B20D635828D15ED02EF8462
S11359A63930628D0CAEE432666E8435108D026E2B
S11359B60434106FE21E034D2A0463E48D1D34463D
S11359C6EE02EC844D2A0463648D1030E48D253296
S11359D6646DE02A028D041E03359043531E03436F
S11359E653C30001240233411E033930621E038D62
S11359F6031E0339327C3446E6E4A6033DE764A677
S1135A0661E6023DEB64E764A662E6013DEB64E70A
S1135A1664A663E6843DEB64E764A661E6033DABF6
S1135A2664ED64A662E6023DE364ED64A663E60102
S1135A363DE364ED64A662E6033DAB65ED652402D1
S1135A466C64A663E6023DE365ED6524026C64A618
S1135A5663E6033DAB66ED6632643546C9008900EC
S1135A66391E3043531E304353C3000124023341CD
S1135A763934063278EC68C3000344564456C300EE
S1135A8601ED66FC7F06ED6210830000260F8E7F13
S1125A9602AF62BF7F06BF7F025F4FED02ECF8E5
S1135AA502EDE4AEE4EC0210A3662539EC0210A382
S1135AB5662607ECF4EDF802201EEEE4EC42A3663C
S1135AC5ED42AEE4EC025849584934061F10E3E1AF
S1135AD5EDE4EC66AEE4ED02EC62FD7F06ECE4C3B6
S1135AE50004326A39ECE410B37F062629EC6658C3
S1135AF5495849BD6555ED641083FFFF26055F4F81
S1135B05326A39EC66AE64ED02EC64C30004BD5B35
S1135B152FFC7F06EDE4ECE4ED62ECF4EDE416FF16
S1135B25823406ECE4BD5A7735903406327CEC6455
S1135B35C3FFFCEDE4FC7F06ED62ECE410A36223F5
S1135B450610A3F802251CEC6210A3F802250DEC3F
S1135B55E410A362220D10A3F8022507ECF802ED68
S1135B656220D7AEE4EC0258495849E3E410A3F89F
S1135B750226141F13EC42AEF802E302ED42AEF81E
S1135B8502EC84EDF42005ECF802EDF4AE62EC02CF
S1125B9558495849E36210A3E426111F13EC4248
S1135BA4AEE4E302ED42ECF4EDF8022005ECE4ED9E
S1135BB4F802EC62FD7F063266393406327E5F4FAA
S1135BC4EDE4AEF802E6844FBD57C5ED7E2720EC24
S1135BD4E4340658495849E3E158493406AEF80414
S1135BE4E680AFF8044FE3E1C3FFD0EDE420D3EC47
S1135BF4E4326439340632E9FEDCAEE90128E68095
S1135C04AFE90128E7E8115D10270668E6E811C149
S1135C1425270CAEE90124E780AFE9012420DBEC5D
S1135C24E90128EDE81EECE9012AEDE82030E82436
S1135C34AFE81ACC0006EDE8156FE818C620E7E8CB
S1135C44196FE817E6F90128C12D2610ECE901289B
S1135C54C30001EDE90128C601E7E818E6F90128C3
S1135C64C1302610ECE90128C30001EDE90128C67E
S1135C7430E7E819E6F90128C12A261AECE90128D3
S1135C84C30001EDE90128AEE9012AEC81AFE90181
S1125C942AEDE813200C30E901281F10BD5BBE78
S1135CA3EDE813E6F90128C12E1026004FC601E7DB
S1135CB3E817ECE90128C30001EDE90128E6F9013D
S1135CC328C12A261AECE90128C30001EDE90128B9
S1135CD3AEE9012AEC81AFE9012AEDE815201DE6BE
S1135CE3F901284FBD57C5ED7E270E30E901281F62
S1135CF310BD5BBEEDE81520036FE817AEE901287C
S1135D03E680AFE90128E7E8116F644FBD667510BB
S1135D1383006C2611C601E764AEE90128E680AF6F
S1135D23E90128E7E811E6E8114FBD6675C063C1D0
S1135D3315102205134F8E5D4058496E9B610C600C
S1135D43035F0F5E155D6C624B624B624B624B6289
S1135D534B624B624B60BA624B624B624B612A6289
S1135D634B605D624B624B608CAEE9012AEC02EE40
S1135D7384ED67EF65BD4BE500000000102700923A
S1135D835F4FED6DEC67EE65BD4BE5000000002C45
S1125D93066C6E26026C6DECE81527066C6E2606
S1135DA2026C6DEC6DE3E815ED6DEC67EE65BD63B9
S1135DB211BD5728BD4FF03E9A209BBD49E23F00DA
S1135DC20000BD4F96EDE82210830000102D013D26
S1135DD2C3FFFF108300092F05CC00052003CC006C
S1135DE204E36DED6FEC67EE65BD4BE53F800000AB
S1135DF22C13EC67EE65BD4BE5BF8000002F066CEB
S1135E026E26026C6DEC6DE3E822ED6D10A36F104B
S1135E122C00FAAEE9012AEE81EC81AFE9012AED08
S1135E2267EF65306B3410306B3410ECE8193406CC
S1135E32EC6DEE6BBD465D3266EDE81C30E824AFD6
S1135E42E81AE6F81C4FBD57A9ED7E10260323EC91
S1135E526B270AC62DAEE81AE780AFE81AEC691080
S1135E628300002E0CC630AEE81AE780AFE81A2091
S1135E7232EC69108300002F2AE6F81C260CC63087
S1135E82AEE81AE780AFE81A2010AEE81CE680AF4D
S1125E92E81CAEE81AE780AFE81AEC6983000158
S1135EA1ED6920CEECE815270AC62EAEE81AE78084
S1135EB1AFE81AEC69108300002C24ECE815108378
S1135EC100002F1BC630AEE81AE780AFE81A6C6AEF
S1135ED126026C69ECE815830001EDE81520D4E68F
S1135EE1F81C2712AEE81CE680AFE81CAEE81AE7FE
S1135EF180AFE81A20E96FF81A30E8241F10BD6654
S1135F01173406ECE815A3E1EDE8131602AAAEE98D
S1135F11012AEE81EC81AFE9012AED67EF65306B6F
S1135F213410306B3410ECE819C300013406EC6D05
S1135F31EE6BBD463E3266EDE81C30E824AFE81A4C
S1135F41E6F81C4FBD57A9ED7E10260226EC6B27FF
S1135F510AC62DAEE81AE780AFE81AAEE81CE6805F
S1135F61AFE81CAEE81AE780AFE81AECE815270A97
S1135F71C62EAEE81AE780AFE81AE6F81C2712AE7F
S1135F81E81CE680AFE81CAEE81AE780AFE81A2007
S1125F91E9C665AEE81AE780AFE81AEC67EE657B
S1135FA0BD4BE5000000002707EC69830001ED69A3
S1135FB0EC69108300002C14C62DAEE81AE780AFFC
S1135FC0E81AEC6940508200ED69200AC62BAEE85D
S1135FD01AE780AFE81ACC000A3406EC6BBD658F73
S1135FE03406344030E8201F10BD6281326630E848
S1135FF0241F10BD66173406ECE815A3E1EDE81381
S11360001601B6E6642712AEE9012AEE81EC81AFEF
S1136010E9012AED62EFE42011AEE9012AEC81AF37
S1136020E9012ABD658FED62EFE4EC62EEE4BD5850
S113603049000000002C1EC62DAEE81AE780AFE828
S11360401AEC62EEE4BD5A67ED62EFE4ECE8138308
S11360500001EDE813C60AE7E812160089E6642792
S113606012AEE9012AEE81EC81AFE9012AED62EF7B
S1136070E42011AEE9012AEC81AFE9012ACE000047
S1136080ED62EFE4C60AE7E81216005AE664271246
S1126090AEE9012AEE81EC81AFE9012AED62EF5E
S113609FE42011AEE9012AEC81AFE9012ACE000018
S11360AFED62EFE4C610E7E812202CE6642712AE87
S11360BFE9012AEE81EC81AFE9012AED62EFE420D8
S11360CF11AEE9012AEC81AFE9012ACE0000ED629D
S11360DFEFE4C608E7E812E6E8124F3406EC64EE84
S11360EF623406344030E8201F10BD628132664F9F
S11360FF3406ECE815A3E1EDE8131600ADAEE901A3
S113610F2AEC81AFE9012AAEE81AE780AFE81AEC6E
S113611FE813830001EDE81316008FE6E81726064F
S113612FCC0100EDE815AEE9012AEC81AFE9012AB3
S113613FEDE81CE6F81C10270070ECE8151027009A
S113614F69AEE81CE680AFE81CAEE81AE780AFE85A
S113615F1AECE815830001EDE815ECE81383000150
S113616FEDE81320CEEC6B2705CC002D2003CC00DB
S113617F2BAEE81AE780AFE81AE6F81C2712AEE850
S112618F1CE680AFE81CAEE81AE780AFE81A20E0
S113619EE96FF81A30E8241F10BD66173406ECE8D0
S11361AE15A3E1EDE813C620E7E8196FF81A30E8F5
S11361BE24AFE81AE6E818263EE6E819C13026169A
S11361CEE6F81AC12D260FE680AFE81AAEE90124CF
S11361DEE780AFE90124ECE813830001EDE813C373
S11361EE0001108300002F0FE6E819AEE90124E741
S11361FE80AFE9012420DFAEE81AE680AFE81AE7A3
S113620EF901245D270DECE90124C30001EDE90138
S113621E2420E4E6E8181027F9D6ECE813830001ED
S113622EEDE813C3000110830000102FF9C2E6E855
S113623E19AEE90124E780AFE9012420DDECE81E64
S113624EEDE90128ECE820EDE9012AE6F901281030
S113625E27F99DAEE90128E680AFE90128AEE901F0
S113626E24E780AFE9012416F9866FF9012432E997
S113627E0126393406327DECF803EDE4EC6BBD6592
S112628E8F34063440EC6DEE6BBD59533264E728
S113629D62C10A2405CB304F2006E6624FC3003796
S11362ADAEF803E780AFF803EC6BBD658F340634AD
S11362BD40EC6DEE6BBD593C3264ED69EF67BD6624
S11362CDB7272EEC6BBD658F34063440EC6DEE6B49
S11362DDBD59533264E762C10A2405CB304F200601
S11362EDE6624FC30037AEF803E780AFF80316FF3D
S11362FDB7AEF8036F84ECE4BD6521ECF803A3E4B9
S113630D4F32653934063440327CEC66EE64ED620E
S113631DEFE4ECE45849EDE4E6E44FC3FF81326861
S113632D39340632E9FF0030E901043410ECE90197
S113633D02340630641F10BD5BF8326430E41F1064
S113634DBD650132E90102393406CC00023406EC94
S113635D62BD63643264393404327D6F62EC66105D
S113636D8300021026007DF6CC222611F6CC2427BC
S113637D0CFCCC24ED66C601E762160078E663C119
S112638D0A260EBDCD245F4FFD7F08CC000132E0
S113639C6439E663C1092638FC7F083406CC00084E
S11363ACBD459F3406CC0008A3E1EDE4FC7F08E373
S11363BCE4FD7F08ECE4830001EDE4C30001ED7E11
S11363CC2708CC0020BD64FB20EACC0001326439E0
S11363DCFC7F08C30001FD7F08E6634FBD64FBCC62
S11363EC0001326439EC66108300032609E6634F1E
S11363FCBD64DD326439AE66E602C101260AC612FA
S113640CE701CCFFFF3264396FF806AE66E6883BD1
S113641CC1FF102700ABE663C10A261BC60DE76358
S113642CE66227085F4FFD7F081600955F4FAE6646
S113643CED89014216008AE663C10910260066E65E
S113644C622705FC7F082006AE66EC8901423406FF
S113645CCC0008BD459F3406CC0008A3E1EDE4E66E
S113646C62270AFC7F08E3E4FD7F08200CEE66EC4F
S113647CC90142E3E4EDC90142C620E763ECE483BD
S112648C0001EDE4C30001108300012F34CC00A4
S113649B203406EC68BD4FCE32621083FFFF26DE3C
S11364ABCCFFFF326439E662270BFC7F08C3000183
S11364BBFD7F08200DAE66EC890142C30001ED8916
S11364CB01426FF806E6634F3406EC68BD4FCE32DB
S11364DB66393406327FF6CC22E7E4C601F7CC22C8
S11364EBEC61BD6355E6E4F7CC22CC000132633991
S11364FB1F98BDCD18393406E6F42715AEE4E680B3
S113650BAFE44FBD63551083FFFF26ECCCFFFF3583
S113651B90CC000135903406327BEC65EDE4BD661E
S113652B173406EC62E3E1ED62ECE410A36224178A
S113653BE6F4E764AE62E682AF62AEE4E780AFE412
S113654BE664E7F80220E23267393406ECE4F36DD3
S113655B52BD656135903406327EEC62C307D03090
S113656B62341010A3E12506CCFFFF326439FC6DB5
S113657B52EDE4EC62FD6D52ECE43264391F01A67A
S112658B637ECD33CE00004D2A02335F393406D0
S113659A30663410EC663406EC64BD5BF832663956
S11365AA340630663410EC663406EC64BD531D328E
S11365BA66393406EC643406EC62BD6617E362BDE0
S11365CA65FB3262ECE435903406AE64E680AF646F
S11365DAE1F4260EAEE4E680AFE4C10026EC5F4F98
S11365EA3590AE64E61F4F3406E6F8024FA3E13550
S11365FA903406327EEC62EDE4AE66E680AF66AEB7
S113660A62E780AF625D26F1ECE432643934063223
S113661A7EEC62EDE4E6F42709ECE4C30001EDE460
S113662A20F3ECE4A3623264393406EC6626045F90
S113663A4F3590AE64E680AF64E1F4261FEC6683BE
S113664A0001ED661083000026045F4F3590AEE426
S113665AE680AFE4C10026DB5F4F3590AE64E61FE7
S113666A4F3406E6F8024FA3E135903404E6E44FCA
S113667ABD5808ED7E2708E6E44FC300202003E650
S112668AE44F4F3261393404E6E44FBD57DAED83
S11366997E2708E6E44FC3FFE02003E6E44F4F32C8
S11366A9613934401E03847F1E038D0235C0118372
S11366B9000026081083000027021CF7393406322B
S11366C9E9FEBCCC0001340630623410ECE901481F
S11366D9BD4D8832641083FFFF2608CCFFFF32E9E1
S11366E9014639FCD409EDE90140ECE90140BD67F3
S11366F95CEDE90140ED7E2746AEE90140EC881CDA
S1136709EDE90142341030621F10BD676D3262ED4C
S11367197E2721C604E7F901405F4F3406ECE901FD
S113672942BD4FCE32621083FFFF2608CCFFFF32F1
S1136739E9014639ECE90142EDE9014016FFABC62E
S11367490CE7E45F4F340630621F10BD4FCE32E9C7
S11367590148393406ECE426045F4F3590ECE4C370
S1136769FFE435903406327DAE63E60FE7E4AE67A5
S1136779E60FE7616F0F5FAE63E70F6F62AE63E623
S112678903AE67E1032632EC67C300043406EC69
S113679865C30004BD65D2326210830000261BEC79
S11367A867C3000C3406EC65C3000CBD65D23262C5
S11367B8108300002604C601E762E6E4AE63E70F2F
S11367C8E661AE67E70FE6624F326539AE628D0A5D
S11367D8C607A6E0A7805A26F939327B1E036FE460
S11367E85849E76366E41F895D2735C1FF271843C5
S11367F86663C07F1D1CF03401ED621F30EE66ED48
S1136808656F6735016EC4CC7FFF6463260C118302
S1136818000026061CF01A0120DD1CF01A0820D7F7
S1136828CC80006463260C1183000026061CF01A31
S11368380420C4CCFF811E0358496963335F2AF8D6
S11368481E0320B11F013007C607A682A7E25A26F5
S1136858F98D0139EC6310837FFF27641083007F6F
S11368682E651083FF812D3ACB7F1F98E668C1807F
S1136878251F2206E667C50127176C6726136C6671
S1126888260F6C65260B4C81FF273C67656666FF
S11368976667E66558686246561F03EC66AEE432DF
S11368A7696E841083FF6A2D1CCB7F6465666666F8
S11368B767A6684624028A01A7685C26EE1F98200B
S11368C7AC86FF20CD4F200286FF6F656F666F672A
S11368D720C07CCC22BDCD247FCC2210FECC2B1033
S11368E78E7E703322CC0001EDA4BDCD27810D2708
S11368F732B1CC02272D812027F05FA7C05CBDCD24
S113690727810D2709B1CC022704812026ED6FE2E8
S1136917A6C2A7E25A26F910EFC1ECA4C30001ED01
S1136927A420C76FE26FE2344010ACE12406ECC345
S1136937340620F36FE210EF6130613410ECA434B5
S113694706307E34108E7E70ACE424046F8020F809
S113695735063506BD45807ECD033406327CEC6AA8
S113696710830001260CEC683406EC66BD69CF324F
S11369776839EC64ED62EC68830001ED681083000C
S1126987002F1BEC6ABD525EEDE41083FFFF2767
S11369960EE661AE62E780AF62C10A270220D86FB5
S11369A6F802ECE41083FFFF260BEC6410A36226C6
S11369B6045F4F2002EC643266393406CC0100349D
S11369C606EC62BD69CF3264393406327AF6CC23DA
S11369D610260043F6CC261027003CFCCC263406B1
S11369E6EC6C3406EC6ABD696132641083000026DF
S11369F6055F4F326839EC66BD6617C3FFFFEDE4E9
S1136A06EC66AEE4E68BC10A26081F10AE66308B30
S1136A166F84EC66326839EC66ED62EC6AED64EC20
S1136A2664830001ED6410830000102F0088BD52BA
S1136A363FEDE41083FFFF1027007BE661C10A26C1
S1136A4609CC000DBD635516006CE661C10D26091F
S1136A56CC000ABD635516005DE661F1CC00263311
S1136A666C6526026C64EC62C3FFFF10A3661025F6
S1136A76FFADEC62830001ED62F6CC07C10826097E
S1126A86CC7E68BD650116FF96F6CC074FBD6345
S1136A955516FF8CE661F1CC012611CC7E6BBD65E4
S1136AA501EC66ED62EC6AED6416FF74E661AE62B4
S1136AB5E780AF6216FF696FF802ECE41083FFFF0D
S1136AC5260BEC6610A36226045F4F2002EC6632A7
S1056AD568391A
S1136CD577940002779A000377A1000477A600054C
S1136CE577AB000677B9000777C1000877CA0009B2
S1136CF577CE000A77D5000B77DF000C77F0000D0F
S1136D0577FD000E7803000F781100107819001133
S1136D157821001278310013783D0014784300156A
S1136D2578530016785E001778640018786C0000B4
S1136D35790C792D794D796D798C79AB79C979E9A6
S1126D45012C000204B000010000000000969C25
S1137E434E6F207375636820746F706963000A252D
S1137E53730A000A00696E66004E614E2830293A9F
S1107E6330303030002008000A3F3F3F005F
S90368D9BB
